:020000040800F2
:1000000000500020C96900085D59000861590008C6
:1000100065590008695900086D5900080000000082
:1000200000000000000000000000000071590008FE
:10003000755900080000000079590008553D000876
:10004000116A0008116A0008116A0008116A0008A4
:10005000116A0008116A0008116A0008116A000894
:10006000116A0008116A0008116A0008116A000884
:10007000116A0008116A0008116A0008116A000874
:10008000116A0008116A0008116A0008116A000864
:10009000116A0008116A0008116A0008116A000854
:1000A000116A0008592D0008116A0008116A000839
:1000B000116A0008116A0008116A0008116A000834
:1000C000116A0008116A0008116A0008116A000824
:1000D000116A000829360008116A0008AD360008C8
:0C00E0007D2E0008116A0008116A00085B
:1000F0000348044B834202D0034B03B118477047B7
:1001000090000020900000200000000005480649F3
:100110000B1AD90F01EBA301491002D0034B03B115
:100120001847704790000020900000200000000059
:1001300010B5064C237843B9FFF7DAFF044B13B12F
:100140000448AFF300800123237010BD900000200D
:1001500000000000146A000808B5044B1BB10449F4
:100160000448AFF30080BDE80840CFE7000000007E
:1001700094000020146A000870B50D4E0D4D761BDA
:10018000B61006D0002455F8043B01349847A64227
:10019000F9D1094E094D06F03DFC761BB61006D08C
:1001A000002455F8043B01349847A642F9D170BDAC
:1001B000B86B0008B86B0008BC6B0008B86B00088F
:1001C000830730B548D0541E002A3FD00346CAB238
:1001D00001E0013C3AD303F8012B9D07F9D1032C30
:1001E0002DD9CDB245EA05250F2C45EA054536D96E
:1001F000A4F1100222F00F0C03F1200EE6444FEAA6
:10020000121C03F1100242E9045542E90255103272
:100210007245F8D10CF1010214F00C0F03EB02123D
:1002200004F00F0C13D0ACF1040323F003030433E8
:10023000134442F8045B9342FBD10CF003042CB14D
:10024000CAB21C4403F8012B9C42FBD130BD64466A
:100250001346002CF4D1F9E703461446BFE71A46CB
:10026000A446E0E70EB410B5044683B008B1836934
:100270005BB106AB2046059AA168019300F014FA21
:1002800003B0BDE8104003B0704700F013F9F0E789
:100290000FB410B50A4B82B01C680CB1A3695BB1F6
:1002A00005AB2046049AA168019300F0FDF902B065
:1002B000BDE8104004B07047204600F0FBF8EFE7BF
:1002C0000000002000207047014900F033B900BF52
:1002D0000111000800207047682270B54D1E02FB16
:1002E00005F50E4605F1740100F048F9044640B1E9
:1002F00000210C30C4E9016005F168022160FFF7BC
:100300005FFF204670BD00BF274B2DE9F0411E68FE
:100310000746B36953B34FF004084836D6E90134B1
:10032000013B04D51EE05A1C04F168041AD0B4F94C
:100330000C50013B002DF6D11C4B08222946C4E984
:100340000055C4E90253C4E904556566A56104F18A
:100350005C00FFF735FFC4E90D55C4E9125520468E
:10036000BDE8F08135682DB12E46D7E7304600F064
:100370001FF8D0E74FF4D671384600F0FFF8044676
:1003800068B1056029460546C0F804800C304FF47A
:10039000D072A060FFF714FF34602E46BEE70C2336
:1003A00030603B60DBE700BF2C6A00080100FFFF04
:1003B0000023334A2DE9F0471268C0E91233904216
:1003C000036508BF01232F4908BF83618162054689
:1003D000FFF79AFF034628466B60FFF795FFA8607A
:1003E00028460024FFF790FF04236E68DFF898A0EA
:1003F000DFF89890DFF89880264FE8600822F360D5
:100400002146C6E90044C6E904447466B460B46198
:1004100006F15C00FFF7D4FE1F4BC6E9086AC6E987
:100420000A983763AE680822F3602146C6E90044A3
:10043000C6E904447466B460B46106F15C00FFF779
:10044000BFFE164BC6E9086AC6E90A983763EE682C
:100450002146F3600822C6E90044C6E904447466F4
:10046000B460B46106F15C00FFF7AAFE0123C6E99F
:10047000086AC6E90B87C6F82890AB61BDE8F0872B
:100480002C6A0008C9020008510D0008790D000807
:10049000B90D0008D90D0008090001001200020082
:1004A000024B0349186800F045B800BF2C6A0008E9
:1004B00001110008836903B97AE77047704700BFEC
:1004C000704700BF704700BF704700BF024B034931
:1004D000186800F00FB800BF00000020C502000837
:1004E000024B0349186800F005B800BF0000002067
:1004F000D50200082DE9F0410026884600F14807A2
:10050000D7E90154013D0ED4A389013D012B06D941
:10051000B4F90E30013302D02046C04706436B1CAD
:1005200004F16804F0D13F68002FE9D13046BDE8FE
:10053000F08100BF2DE9F8434FF0000907468846D7
:1005400000F14806D6E90154013D10D4A389013DCC
:10055000012B08D9B4F90E30013304D021463846B6
:10056000C04749EA00096B1C04F16804EED1366803
:10057000002EE7D14846BDE8F88300BFF8B5CD1C92
:1005800025F0030508350C2D38BF0C25002D064637
:1005900023DBA94221D8264F01F072F93A6822B331
:1005A000144603E063682246FBB11C4623685B1BCC
:1005B000F8D40B2B15D8636894420CBF3B60536092
:1005C000304601F05FF904F10B00231D20F0070015
:1005D000C21A01D01B1AA350F8BD0C2300203360AF
:1005E000F8BD23601C442560EAE77968D1B129464B
:1005F000304600F09BFB431C01460CD0C41C24F089
:100600000304A04205D03046611A00F08FFB013090
:1006100001D02560D4E70C233046336001F032F975
:100620000020F8BD304600F081FB7860DFE700BFB6
:10063000AC0000209368013B002B936005DAD2F8F0
:1006400018C0634507DB0A2905D01368581C1060E1
:1006500008461970704700F0C3BB00BF9BB1F8B5E6
:10066000134406460F46541E5D1E01E0AC4208D0FE
:100670003A46304614F8011FFFF7DCFF431CF5D162
:10068000F8BD0020F8BD0020704700BF936810B58A
:10069000144613B91846536010BD00F09BFD0023AB
:1006A000C4E9013310BD00BF2DE9F04F0E4692465C
:1006B0001C4607469FB018B18369002B00F0A88044
:1006C000954B9E4200F0AA80944B9E4200F0B5806C
:1006D000934B9E4208BFFE68B389180740F1A38080
:1006E0003369002B00F09F80002320220B933023DE
:1006F0009AF80010059401258A4C8DF831208DF868
:10070000323000297DD0D1460B4604E019F8013F74
:10071000002B00F09480252BF8D1B9EB0A0B40F0A8
:10072000918099F80030002B6BD000234FF0FF32FE
:1007300009F10109CDE90723069309938DF85B3090
:100740001C9304E0001B05FA00F018430690CA460B
:100750000522204619F8011B00F058FF069B0028CF
:10076000F0D1D90644BF20228DF85B201A0748BF7C
:100770002B229AF8001048BF8DF85B202A2972D1ED
:10078000059A1168043200290592C0F2A0800991EF
:100790009AF801100AF1010A2E2976D0DFF8889123
:1007A0000322484600F032FF48B14022069BA0EBEE
:1007B000090002FA00F003430AF1010A06931AF84D
:1007C000011B062259488DF8301000F01FFF002849
:1007D00000F08380564B002B6CD005A90091324667
:1007E0003846544B06A9AFF300800390039B0133B6
:1007F00007D00B9B039A9AF8001013440B9300291F
:1008000081D1B3895B0615D40B981FB0BDE8F08F7A
:10081000FFF750FE404B9E427FF456AF7E68B3898F
:1008200018073FF55DAF3146384600F051FB002810
:100830003FF45AAF4FF0FF30E7E7BE684CE7B9EB43
:100840000A0BDED0D046CAF1010A03E0934538D93D
:1008500018F8011F32463846FFF7ECFE01300AEB6C
:100860000802F3D1CDE7A1F13002092A94D8099BFF
:100870001AF8011F03EB830302EB4303A1F13002DB
:10088000092AF5D92E29099388D19AF801102A2925
:100890002DD1059B0AF102001A680433002A059342
:1008A000B8BF4FF0FF339AF8021007928246B8BFE4
:1008B000079373E7059B073323F00703083305937A
:1008C00097E70B9A99F800305A440B922BE749426C
:1008D00043F00203099106935AE705A900913246B5
:1008E0003846144B06A900F0CBF803907EE70023AE
:1008F000A1F13002092A0AF1010A07933FF64EAF2F
:100900001AF8011F03EB830302EB4303A1F130024A
:10091000092AF5D9079341E7706A0008506A000870
:10092000306A00087C6B0008846B0008886B000844
:10093000000000005D0600088C4600B586461346A0
:10094000034A714610685DF804EB6246FFF7ACBEDF
:10095000000000202DE9F04791461E460A698B6889
:100960000C469A42B8BF1A46C9F8002091F84330A5
:100970000546DDF8208013B10132C9F80020226855
:1009800091065DD5D9F800300233C9F800302268ED
:1009900012F0060F11461ED1E168CB1A002BD8BF0A
:1009A000114618DD002704F1190A06E0D9F80030D5
:1009B000E268A2EB030CBC450CDD01235246314634
:1009C0002846C047013007F10107EFD14FF0FF3053
:1009D000BDE8F087216894F84330003B18BF01233D
:1009E0008A060AD53021E21882F8431094F845109F
:1009F0005A1C2244023382F843103146284604F13F
:100A00004302C0470130E1D0236803F00603042B02
:100A10001DD0A3682269934225DD00279B1A1F443D
:100A200004F11A09002401E0BC421CDA01234A4601
:100A300031462846C047013004F10104F4D1C5E72E
:100A400012F0060F12D0003B18BF0123D5E7D9F8EA
:100A50000030E1682269C91AA36821EAE17793426C
:100A6000DCDC0029DCDC0020BDE8F087E168D9F897
:100A70000030CB1A002BD8BF114693DCABE700BF88
:100A80002DE9F04317460A7E85B00C460646984687
:100A90000C9D01F1430C002A33D0A2F15803D9B2C6
:100AA000202967D8202B65D8DFE813F0DD0064002B
:100AB0006400640064006400640064006400640016
:100AC0006400A3006E0064006400640064006E00B3
:100AD000640064006400640021007F00BF006400C3
:100AE0006400AE0064007F0064006400E4002368DA
:100AF0001A0640F102812B686269191D29601B6882
:100B00001A600023E14623613B4621463046CDF87A
:100B1000008003AAFFF71EFF013020D04A46394665
:100B200030462369C047013019D02368E0689B072D
:100B3000039919D5431A002B16DD002504F1190974
:100B400004E0E0680399431AAB420DDD01234A46F5
:100B500039463046C047013005F10105F1D14FF06B
:100B6000FF3005B0BDE8F0838842B8BF084605B045
:100B7000BDE8F083012384F8422004F14209236197
:100B8000002384F84330BFE72368190602D45A06CD
:100B900000F1BF8029680A68043129601146002AE3
:100BA0006ADB0A25DFF87CE110E02368180640F1D3
:100BB0009A802B68191D296019686F2A0CBF0825B7
:100BC0000A25DFF860E1002384F843306268002AD8
:100BD000A2607DDB236823F004032360002959D140
:100BE000002A77D1E146082D63D0ACEB09032361DD
:100BF0008AE701222B6804F14209196804332B604B
:100C000084F842102261BBE72B6800211A1D2A607C
:100C1000D3F800906268484600F0F8FC00287FD0C6
:100C2000A0EB090060602061AAE7236843F020037D
:100C300023607822DFF8F0E084F845202A68111D4F
:100C40002960190642D45D0640D51188D80744BFF3
:100C500043F020032360002943D12368102523F0AB
:100C600020032360AFE75823DFF8B8E084F845306D
:100C70002368E3E72368DCE72D2284F843206268D9
:100C80004942002AA26002DB23F0040323600A2504
:100C9000DFF890E0E146B1FBF5F30A4605FB1310DF
:100CA00019461EF80030AA4209F8013DF3D2082D7A
:100CB0009BD12368D90798D5626823699A4294DC4E
:100CC000302309F1FF3989F800308EE71168BDE75C
:100CD0000029DFD19EF8003004F1420984F8423047
:100CE00081E710256FE713F0400F2B6803F1040133
:100CF00029600CBF196819885FE713F0400F2B6853
:100D0000626903F1040129601B6814BF1A801A602C
:100D1000F7E62A68B2F9001004322A600A463EE774
:100D2000606880E7906B0008A46B0008002238B56B
:100D3000064D044608462A6001F0B2FD431C00D06F
:100D400038BD2B68002BFBD0236038BDB4000020D9
:100D500010B50C46B1F90E1000F024FE002803DB9C
:100D6000636D0344636510BDA38923F48053A3819D
:100D700010BD00BF002070472DE9F0410C46B1F9CD
:100D80000C101F46CB05054616460BD421F48051A6
:100D9000A1813B4632462846B4F90E10BDE8F04129
:100DA00000F080B8B4F90E100223002200F08AFB94
:100DB000B4F90C10EAE700BF10B50C46B1F90E10FB
:100DC00000F080FBA389421C0EBF23F4805343F440
:100DD00080536065A38110BDB1F90E1000F0FAB820
:100DE000F8B506460D46144608B1836943B3254B52
:100DF0009C422AD0244B9C4229D0244B9C4208BFC1
:100E0000F468A269A389A2601A0722D5236903B3F3
:100E100022686169D31AEDB299422F4629DD013368
:100E2000A1680139A160511C2160157062699A4264
:100E300016D0A389DB0701D50A2D11D03846F8BD9D
:100E4000FFF738FB0F4B9C42D4D17468D9E7B468E4
:100E5000D7E72146304600F03BF838B92369D7E799
:100E60002146304600F04CF90028E7D04FF0FF371C
:100E7000E4E72146304600F043F90028F6D101238B
:100E80002268CDE7706A0008506A0008306A0008DE
:100E900003460A46024908681946FFF7A1BF00BF8A
:100EA0000000002038B50C46114600228446074D4C
:100EB00020462A601A46644601F000FD431C00D01B
:100EC00038BD2B68002BFBD0236038BDB400002058
:100ED0003C4B70B51D6806460C460DB1AB69E3B1DD
:100EE000394B9C421FD0394B9C424DD0384B9C42D1
:100EF00008BFEC68B4F90C3018079AB219D521690B
:100F000011B312F001002FD000256069A5604042A6
:100F1000A06100292ED0002070BD2846FFF7CAFA34
:100F2000294B9C42DFD16C68B4F90C3018079AB297
:100F3000E5D4D1063ED5520728D4216943F00803F1
:100F4000A3819AB20029DCD102F42070B0F5007FB1
:100F5000D7D02146304600F0CBFAB4F90C302169E5
:100F60009AB212F00100CFD1950758BF6069A06016
:100F70000029D0D1120658BF0846CDD543F0400312
:100F80004FF0FF30A38170BDAC68B3E7616B51B126
:100F900004F14402914204D0304600F075FCB4F9EB
:100FA0000C30002262630022216923F02403C4E98B
:100FB0000012C3E7092243F0400332604FF0FF30D4
:100FC000A38170BD00000020706A0008506A00080C
:100FD000306A0008002238B5064D044608462A60EB
:100FE00001F036FC431C00D038BD2B68002BFBD031
:100FF000236038BDB4000020F8B58B890C46190772
:1010000007463BD46268002A55DDE66A002E50D0C0
:1010100000223D683A6013F4805250D101233846D3
:10102000216AB047421C5CD0A389E66A5B0705D5FC
:101030006368C01A636B0BB1236CC01A0246216A45
:1010400000233846B047411C3BD13B68002B38D0C9
:101050001D2B01D0162B4BD100232269C4E900239C
:10106000616B3D6029B304F14403994202D03846D4
:1010700000F00AFC002318466363F8BD2669C6B178
:101080009A0718BF0023256808BF63692660AD1B57
:10109000A3600CE02B463246D4F828C03846216ABB
:1010A000E047B0F1000CA5EB0C05664412DD002D05
:1010B000F0DC0020F8BD226C002AA6DCF9E7606DA8
:1010C000B4E70022236962602360A389DB04C7D5EB
:1010D0006065C5E7A3894FF0FF3043F04003A3816B
:1010E000F8BD3B68002B9FD01D2B06D0162B04D0DB
:1010F000A38943F04003A381F8BD00203D60F8BD03
:1011000038B50B69BBB10C46054608B18369B3B16C
:101110000D4B9C4211D00D4B9C4213D00C4B9C426A
:1011200008BFEC68B4F90C302BB121462846BDE865
:101130003840FFF761BF002038BD6C68F2E7FFF769
:10114000B9F9E5E7AC68EDE7706A0008506A000895
:10115000306A000838B540B303690446E3B1174B61
:101160001D680DB1AB69CBB1154B9C420FD0154B2F
:101170009C4221D0144B9C4208BFEC68B4F90C305F
:1011800053B121462846BDE83840FFF735BF6C68AB
:10119000B4F90C30002BF4D1002038BD2846FFF7FD
:1011A00089F9074B9C42E2D1F1E7084B08491868DE
:1011B000BDE83840FFF7BEB9AC68DFE700000020AB
:1011C000706A0008506A0008306A00082C6A00083B
:1011D000011100089368002B00F0B7802DE9F04F53
:1011E000B1F90C300C4619078046174683B098B207
:1011F00025D523691BB310F002033D682DD04FF0B5
:10120000000B5E46DFF8B8A2002E00F08B8056453A
:1012100033465A4628BF53464046216AD4F828C070
:10122000E047002840F38780BB6883441B1A361AC6
:10123000BB60002BE8D1002003B0BDE8F08F214651
:101240004046FFF745FE002840F03681B4F90C30E7
:101250003D6898B210F00203D1D110F0010976D1A7
:101260004E46002E5AD08205D4F808B040F1B58021
:10127000B3455A4600F2CD8010F4906F00F0CB8059
:1012800023682169A3EB010B636903EB430A0AEBB3
:10129000DA7A0BF101034FEA6A0A334453455246A6
:1012A00084BF9A465246430540F1EA8011464046C3
:1012B000FFF764F9002800F0F9805A46216901908F
:1012C00000F0ECF9A289019B22F4906242F08002C6
:1012D000A28103EB0B0023613246AAEB0B03B3465A
:1012E000C4F814A0A3602060B246002649460192CB
:1012F00000F04AFAA3682168019AA3EB0B030A44A1
:10130000A3602260B868D144A0EB0A00B86000284E
:1013100091D0B4F90C0080B2002EA4D1D5E900968A
:1013200008359EE7D5E900B608356DE72146404609
:10133000FFF7E6FE80B3B4F90C304FF0FF3043F016
:101340004003A38103B0BDE8F08F002070471E4624
:10135000AA46994618461D4656B3002832D04A463A
:1013600020682169B24228BF32468842636904D9A5
:10137000A16803EB010B5A4574DC934265DC2A46F5
:101380004046216AD4F828C0E047B0F1000BD2DD16
:10139000B9EB0B09CAD00120BB685D44A3EB0B037A
:1013A000A6EB0B06BB60002B3FF445AF002ED4D15B
:1013B0000AF1080353F8046C9A4653F8085C0833A2
:1013C000002EF7D032460A21284600F01FF90028E7
:1013D00069D00130A0EB0509C1E720682369984274
:1013E0001BD86369B34218D86FF0004CB44528BFCE
:1013F000B4469CFBF3FC4A4603FB0CF34046216ACF
:10140000D4F828C0E047B0F1000A94DDA6EB0A0644
:1014100078E7B3463246206866E7B345DA4628BF28
:10142000B2464946524600F0AFF9A3682268A3EBE2
:101430000A035244A3602260002BE7D121464046B4
:10144000FFF75EFE0028E1D075E72946934601923A
:1014500000F09AF9A368019A9B1AA36023681A44C2
:10146000226095E729465A4600F08EF92368214606
:101470005B4440462360FFF743FE002888D05AE7CC
:10148000404600F067FA034600287FF422AF40464A
:10149000216900F0F9F90C22B4F90C30C8F80020E9
:1014A00023F0800349E7721C914659E70C22B4F9F6
:1014B0000C30C8F8002040E74FF0FF30BCE600BF1A
:1014C00000FCFF7F38B50C46114600228446074DCC
:1014D00020462A601A46644601F0D2F9431C00D027
:1014E00038BD2B68002BFBD0236038BDB400002032
:1014F000F0B58B890C46990797B007D5012204F106
:101500004703C4E90432236017B0F0BDB4F90E10EC
:10151000054600292DDB6A4600F05AFA002827DB31
:10152000019E4FF4806706F47046A6F50056B6FAA1
:1015300086F6394628467609FFF720F830B3A389A6
:101540001A4A43F08003AA62C4E90407A381206019
:10155000002ED9D02846B4F90E1000F04DFA00281C
:10156000D2D0A38923F0030343F00103A381CBE787
:10157000A38913F0800F14BF40274FF480672846DB
:1015800039460026FEF7FAFF0028D8D1B4F90C300E
:101590009A05B9D4012123F0030304F1470243F073
:1015A0000203C4E90421A3812260ADE7C902000857
:1015B00070B50C46B1F90E10164600291D4696B0BE
:1015C00013DB6A4600F004FA00280EDB01994FF4A1
:1015D000806301F47041A1F50051B1FA81F100205E
:1015E00049092960336016B070BD0022B4F90C308F
:1015F0002A601B0604D540230020336016B070BD5E
:101600004FF480630020336016B070BD5FFA81FC38
:10161000810710D00346511E2AB90AE09A071846DE
:101620000AD0013905D3184613F8012B6245F5D1CC
:10163000704700207047114603290CD80029F8D0C4
:101640000346014401E08B42F3D0184613F8012B06
:101650006245F8D1ECE7024610B54CEA0C2444EAA6
:1016600004441046036804326340A3F1013E2EEAAD
:10167000030313F0803F04D1043903291046F0D846
:1016800051B10346014401E08B4205D0184613F8DE
:10169000012B6245F8D110BD002010BD844641EAFF
:1016A000000313F0030349D1403A23D30B680360CE
:1016B0004B6843608B688360CB68C3600B690361D0
:1016C0004B6943618B698361CB69C3610B6A0362B8
:1016D0004B6A43628B6A8362CB6AC3620B6B0363A0
:1016E0004B6B43638B6B8363CB6BC3634030403185
:1016F000403ADBD230320BD30B6803604B68436057
:101700008B688360CB68C36010301031103AF3D21D
:101710000C3205D351F8043B40F8043B043AF9D2AB
:10172000043208D0D2071CBF11F8013B00F8013B7E
:1017300001D30B8803806046704700BF082A13D38B
:101740008B07B1D010F00303AED0C3F10403D21A5B
:10175000DB071CBF11F8013B00F8013BA4D331F8B3
:10176000023B20F8023B9FE7043AD9D3013A11F833
:10177000013B00F8013BF9D20B7803704B784370C2
:101780008B7883706046704788420DD98B188342EE
:101790000AD900EB020CBAB1624613F801CD9942A6
:1017A00002F801CDF9D170470F2A0ED8034602F195
:1017B000FF3C4AB10CF1010C013B8C4411F8012BA8
:1017C000614503F8012FF9D1704740EA01039B07F7
:1017D0004FD1A2F1100370B501F1200C23F00F05D9
:1017E00001F1100E00F11004AC441B095EF8105C0E
:1017F0000EF1100E44F8105C5EF81C5C103444F8D6
:101800001C5C5EF8185C44F8185C5EF8145CE645F5
:1018100044F8145CEAD1013312F00C0F01EB031110
:1018200002F00F0400EB031327D08E46043C24F093
:1018300003064FEA940C1E441C1F5EF8045B44F838
:10184000045FB442F9D10CF1010402F0030203EB8E
:10185000840301EB840102F1FF3C4AB10CF1010C5D
:10186000013B8C4411F8012B614503F8012FF9D19C
:1018700070BD034602F1FF3C9CE72246EBE700BF48
:10188000704700BF704700BF002952D038B551F8EB
:10189000043C0C1F002BB8BFE4180546FFF7F0FF0F
:1018A0002B4A1368002B45D0A3420CD9216860183D
:1018B000834228D0636028461460BDE83840FFF7B3
:1018C000E1BFA3420FD81A465B68002BF9D111681B
:1018D000501884421DD034D3636054602846BDE85C
:1018E0003840FFF7CFBF11685018A04215D028D854
:1018F000216860188342EFD118685B680144C4E92D
:1019000000135460EAE718685B680144C4E90013F7
:10191000D1E7236819441160E0E7206801445018BA
:1019200083421160DAD1D3E900030144C2E9001314
:10193000D4E77047284663601460BDE83840FFF77D
:10194000A1BF0C2328462B60BDE83840FFF79ABFA3
:10195000AC000020F8B51446F9B1CAB106460D46F0
:1019600000F05CF8A04202D32F463846F8BD21466D
:101970003046FEF703FE07460028F6D022462946E9
:10198000FFF78CFE30462946FFF77EFF3846F8BD4C
:101990002746FFF779FF3846F8BD1146BDE8F84005
:1019A000FEF7ECBD38B50C46114600228446074DC3
:1019B00020462A601A46644600F06AFF431C00D0A5
:1019C00038BD2B68002BFBD0236038BDB40000204D
:1019D00070B50026074D0446084611462E6000F0FB
:1019E0003FFF431C00D070BD2B68002BFBD0236051
:1019F00070BD00BFB4000020002238B5064D04467B
:101A000008462A6000F034FF431C00D038BD2B6824
:101A1000002BFBD0236038BDB400002051F8040C2B
:101A20000028A0F10400BCBF0B58C018704700BFCD
:101A300081F0004102E000BF83F0004330B54FEA7F
:101A400041044FEA430594EA050F08BF90EA020FEC
:101A50001FBF54EA000C55EA020C7FEA645C7FEA7F
:101A6000655C00F0E2804FEA5454D4EB5555B8BFA2
:101A70006D420CDD2C4480EA020281EA030382EA13
:101A8000000083EA010180EA020281EA0303362DA5
:101A900088BF30BD11F0004F4FEA01314FF4801C78
:101AA0004CEA113102D0404261EB410113F0004F8A
:101AB0004FEA03334CEA133302D0524263EB430341
:101AC00094EA050F00F0A780A4F10104D5F1200EDF
:101AD0000DDB02FA0EFC22FA05F2801841F100013A
:101AE00003FA0EF2801843FA05F359410EE0A5F10E
:101AF00020050EF1200E012A03FA0EFC28BF4CF03F
:101B0000020C43FA05F3C01851EBE37101F00045F4
:101B100007D54FF0000EDCF1000C7EEB00006EEB01
:101B20000101B1F5801F1BD3B1F5001F0CD349088B
:101B30005FEA30004FEA3C0C04F101044FEA4452E2
:101B400012F5800F80F09A80BCF1004F08BF5FEA69
:101B5000500C50F1000041EB045141EA050130BD49
:101B60005FEA4C0C404141EB0101013C28BFB1F55B
:101B7000801FE9D291F0000F04BF01460020B1FAA6
:101B800081F308BF2033A3F10B03B3F120020CDA79
:101B90000C3208DD02F1140CC2F10C0201FA0CF057
:101BA00021FA02F10CE002F11402D8BFC2F1200CBC
:101BB00001FA02F120FA0CFCDCBF41EA0C01904072
:101BC000E41AA2BF01EB0451294330BD6FEA0404BB
:101BD0001F3C1CDA0C340EDC04F11404C4F12002A6
:101BE00020FA04F001FA02F340EA030021FA04F3B8
:101BF00045EA030130BDC4F10C04C4F1200220FA0F
:101C000002F001FA04F340EA0300294630BD21FA4C
:101C100004F0294630BD94F0000F83F4801306BF12
:101C200081F480110134013D4EE77FEA645C18BF06
:101C30007FEA655C29D094EA050F08BF90EA020F9D
:101C400005D054EA000C04BF1946104630BD91EA95
:101C5000030F1EBF0021002030BD5FEA545C05D198
:101C60004000494128BF41F0004130BD14F58004D7
:101C70003CBF01F5801130BD01F0004545F0FE414B
:101C800041F470014FF0000030BD7FEA645C1ABF80
:101C9000194610467FEA655C1CBF0B46024650EAB7
:101CA000013406BF52EA033591EA030F41F40021E3
:101CB00030BD00BF90F0000F04BF0021704730B569
:101CC0004FF4806404F132044FF000054FF000013E
:101CD00050E700BF90F0000F04BF0021704730B5FF
:101CE0004FF4806404F1320410F0004548BF4042D4
:101CF0004FF000013EE700BF42004FEAE2014FEA29
:101D000031014FEA02701FBF12F07F4393F07F4F03
:101D100081F06051704732F07F4208BF704793F006
:101D20007F4F04BF41F40021704730B54FF4607419
:101D300001F0004521F000411CE700BF50EA01021C
:101D400008BF704730B54FF000050AE050EA0102C5
:101D500008BF704730B511F0004502D5404261EB35
:101D600041014FF4806404F132045FEA915C3FF476
:101D7000D8AE4FF003025FEADC0C18BF03325FEA13
:101D8000DC0C18BF033202EBDC02C2F1200300FAC4
:101D900003FC20FA02F001FA03FE40EA0E0021FAE9
:101DA00002F11444BDE600BF70B54FF0FF0C4CF4D7
:101DB000E06C1CEA11541DBF1CEA135594EA0C0F89
:101DC00095EA0C0F00F0DEF82C4481EA030621EAC4
:101DD0004C5123EA4C5350EA013518BF52EA0335FF
:101DE00041F4801143F4801338D0A0FB02CE4FF0B1
:101DF0000005E1FB02E506F00042E0FB03E54FF0E1
:101E00000006E1FB03569CF0000F18BF4EF0010ED8
:101E1000A4F1FF04B6F5007F64F5407404D25FEAD4
:101E20004E0E6D4146EB060642EAC62141EA555187
:101E30004FEAC52040EA5E504FEACE2EB4F1FD0CC9
:101E400088BFBCF5E06F1ED8BEF1004F08BF5FEA47
:101E5000500E50F1000041EB045170BD06F00046F9
:101E600046EA010140EA020081EA0301B4EB5C04A6
:101E7000C2BFD4EB0C0541EA045170BD41F480119E
:101E80004FF0000E013C00F3AB8014F1360FDEBFC3
:101E9000002001F0004170BDC4F10004203C35DA9F
:101EA0000C341BDC04F11404C4F1200500FA05F322
:101EB00020FA04F001FA05F240EA020001F00042C3
:101EC00021F0004110EBD37021FA04F642EB060139
:101ED0005EEA430E08BF20EAD37070BDC4F10C0463
:101EE000C4F1200500FA04F320FA05F001FA04F227
:101EF00040EA020001F0004110EBD37041F1000113
:101F00005EEA430E08BF20EAD37070BDC4F120051D
:101F100000FA05F24EEA020E20FA04F301FA05F285
:101F200043EA020321FA04F001F0004121FA04F22D
:101F300020EA020000EBD3705EEA430E08BF20EAFD
:101F4000D37070BD94F0000F0FD101F00046400037
:101F500041EB010111F4801F08BF013CF7D041EAB9
:101F6000060195F0000F18BF704703F000465200BD
:101F700043EB030313F4801F08BF013DF7D043EA8E
:101F80000603704794EA0C0F0CEA135518BF95EA44
:101F90000C0F0CD050EA410618BF52EA4306D1D1CB
:101FA00081EA030101F000414FF0000070BD50EAEA
:101FB000410606BF1046194652EA430619D094EA74
:101FC0000C0F02D150EA013613D195EA0C0F05D15E
:101FD00052EA03361CBF104619460AD181EA0301B2
:101FE00001F0004141F0FE4141F470014FF000006A
:101FF00070BD41F0FE4141F4780170BD70B54FF005
:10200000FF0C4CF4E06C1CEA11541DBF1CEA135584
:1020100094EA0C0F95EA0C0F00F0A7F8A4EB050466
:1020200081EA030E52EA03354FEA013100F088805D
:102030004FEA03334FF0805545EA131343EA126326
:102040004FEA022245EA111545EA10654FEA0026DB
:102050000EF000419D4208BF964244F1FD0404F594
:10206000407402D25B084FEA3202B61A65EB0305F0
:102070005B084FEA32024FF480104FF4002CB6EBAD
:10208000020E75EB030E22BFB61A754640EA0C002D
:102090005B084FEA3202B6EB020E75EB030E22BF6D
:1020A000B61A754640EA5C005B084FEA3202B6EBAE
:1020B000020E75EB030E22BFB61A754640EA9C006D
:1020C0005B084FEA3202B6EB020E75EB030E22BF3D
:1020D000B61A754640EADC0055EA060E18D04FEAFB
:1020E000051545EA16754FEA06164FEAC30343EA9B
:1020F00052734FEAC2025FEA1C1CC0D111F4801F68
:102100000BD141EA00014FF000004FF0004CB6E760
:1021100011F4801F04BF01430020B4F1FD0C88BFFF
:10212000BCF5E06F3FF6AFAEB5EB030C04BFB6EB0A
:10213000020C5FEA500C50F1000041EB045170BDFD
:102140000EF0004E4EEA113114EB5C04C2BFD4EB2A
:102150000C0541EA045170BD41F480114FF0000EAE
:10216000013C90E645EA060E8DE60CEA135594EA2A
:102170000C0F08BF95EA0C0F3FF43BAF94EA0C0F2D
:102180000AD150EA01347FF434AF95EA0C0F7FF4A2
:1021900025AF104619462CE795EA0C0F06D152EAF6
:1021A00003353FF4FDAE1046194622E750EA4106DA
:1021B00018BF52EA43067FF4C5AE50EA41047FF4EB
:1021C0000DAF52EA43057FF4EBAE12E74FEA41024E
:1021D00012F5001215D211D56FF47873B3EB625279
:1021E00012D94FEAC12343F0004343EA505311F0A0
:1021F000004F23FA02F018BF404270474FF0000032
:10220000704750EA013005D111F0004008BF6FF06F
:10221000004070474FF00000704700BF4A0011D2E5
:1022200012F5001211D20DD56FF47873B3EB625230
:102230000ED44FEAC12343F0004343EA505323FA3C
:1022400002F070474FF00000704750EA013002D1B1
:102250004FF0FF3070474FF00000704780F00040B3
:1022600002E000BF81F0004142001FBF5FEA41036E
:1022700092EA030F7FEA226C7FEA236C6AD04FEA6E
:102280001262D2EB1363C1BFD218414048404140B3
:10229000B8BF5B42192B88BF704710F0004F40F465
:1022A000000020F07F4018BF404211F0004F41F481
:1022B000000121F07F4118BF494292EA030F3FD04D
:1022C000A2F1010241FA03FC10EB0C00C3F1200360
:1022D00001FA03F100F0004302D5494260EB4000EF
:1022E000B0F5000F13D3B0F1807F06D340084FEA5A
:1022F000310102F10102FE2A51D2B1F1004F40EB4F
:10230000C25008BF20F0010040EA030070474900B6
:1023100040EB0000013A28BFB0F5000FEDD2B0FA53
:1023200080FCACF1080CB2EB0C0200FA0CF0AABF76
:1023300000EBC25052421843BCBFD0401843704714
:1023400092F0000F81F4000106BF80F4000001321A
:10235000013BB5E74FEA41037FEA226C18BF7FEAF1
:10236000236C21D092EA030F04D092F0000F08BF33
:102370000846704790EA010F1CBF0020704712F01A
:102380007F4F04D1400028BF40F00040704712F159
:1023900000723CBF00F50000704700F0004343F0BE
:1023A000FE4040F4000070477FEA226216BF0846F4
:1023B0007FEA23630146420206BF5FEA412390EAB7
:1023C000010F40F4800070474FF0000304E000BFAD
:1023D00010F0004348BF40425FEA000C08BF70475E
:1023E00043F0964301464FF000001CE050EA010222
:1023F00008BF70474FF000030AE000BF50EA010237
:1024000008BF704711F0004302D5404261EB410123
:102410005FEA010C02BF84460146002043F0B64348
:1024200008BFA3F18053A3F50003BCFA8CF2083A6D
:10243000A3EBC25310DB01FA02FC634400FA02FC76
:10244000C2F12002BCF1004F20FA02F243EB02007D
:1024500008BF20F00100704702F1200201FA02FCDF
:10246000C2F1200250EA4C0021FA02F243EB0200D2
:1024700008BF20EADC7070474FF0FF0C1CEAD05216
:102480001EBF1CEAD15392EA0C0F93EA0C0F6FD0D7
:102490001A4480EA010C400218BF5FEA41211ED0B5
:1024A0004FF0006343EA501043EA5111A0FB0131A1
:1024B0000CF00040B1F5000F3EBF490041EAD37176
:1024C0005B0040EA010062F17F02FD2A1DD8B3F1F2
:1024D000004F40EBC25008BF20F00100704790F061
:1024E000000F0CF0004C08BF49024CEA502040EAB3
:1024F00051207F3AC2BFD2F1FF0340EAC250704779
:1025000040F400004FF00003013A5DDC12F1190FB6
:10251000DCBF00F000407047C2F10002410021FA28
:1025200002F1C2F1200200FA02FC5FEA310040F140
:10253000000053EA4C0308BF20EADC70704792F0B9
:10254000000F00F0004C02BF400010F4000F013AF1
:10255000F9D040EA0C0093F0000F01F0004C02BFEC
:10256000490011F4000F013BF9D041EA0C018FE75B
:102570000CEAD15392EA0C0F18BF93EA0C0F0AD061
:1025800030F0004C18BF31F0004CD8D180EA010087
:1025900000F00040704790F0000F17BF90F0004F20
:1025A000084691F0000F91F0004F14D092EA0C0F02
:1025B00001D142020FD193EA0C0F03D14B0218BF95
:1025C000084608D180EA010000F0004040F0FE40DB
:1025D00040F40000704740F0FE4040F44000704777
:1025E0004FF0FF0C1CEAD0521EBF1CEAD15392EAF6
:1025F0000C0F93EA0C0F69D0A2EB030280EA010CE6
:1026000049024FEA402037D04FF0805343EA11117E
:1026100043EA10130CF000408B4238BF5B0042F1DC
:102620007D024FF4000C8B4224BF5B1A40EA0C0081
:10263000B3EB510F24BFA3EB510340EA5C00B3EBB3
:10264000910F24BFA3EB910340EA9C00B3EBD10FA1
:1026500024BFA3EBD10340EADC001B0118BF5FEAF3
:102660001C1CE0D1FD2A3FF650AF8B4240EBC2501C
:1026700008BF20F0010070470CF0004C4CEA5020DD
:102680007F32C2BFD2F1FF0340EAC250704740F42C
:1026900000004FF00003013A37E792F0000F00F01E
:1026A000004C02BF400010F4000F013AF9D040EA9C
:1026B0000C0093F0000F01F0004C02BF490011F430
:1026C000000F013BF9D041EA0C0195E70CEAD15328
:1026D00092EA0C0F08D142027FF47DAF93EA0C0F0F
:1026E0007FF470AF084676E793EA0C0F04D14B02F3
:1026F0003FF44CAF08466EE730F0004C18BF31F0A5
:10270000004CCAD130F000427FF45CAF31F000439E
:102710007FF43CAF5FE700BF4FF0FF3C06E000BF37
:102720004FF0010C02E000BF4FF0010C4DF804CD5A
:102730004FEA40024FEA41037FEA226C18BF7FEA6A
:10274000236C11D001B052EA530C18BF90EA010F6C
:1027500058BFB2EB030088BFC81738BF6FEAE170FB
:1027600018BF40F0010070477FEA226C02D15FEA97
:10277000402C05D17FEA236CE4D15FEA412CE1D003
:102780005DF8040B704700BF844608466146FFE7CA
:102790000FB5FFF7C9FF002848BF10F1000F0FBDAC
:1027A0004DF808EDFFF7F4FF0CBF012000205DF8A5
:1027B00008FB00BF4DF808EDFFF7EAFF34BF01202A
:1027C00000205DF808FB00BF4DF808EDFFF7E0FFC3
:1027D00094BF012000205DF808FB00BF4DF808ED14
:1027E000FFF7D2FF94BF012000205DF808FB00BF77
:1027F0004DF808EDFFF7C8FF34BF012000205DF859
:1028000008FB00BF4FEA4002B2F1FE4F0FD34FF07A
:102810009E03B3EB12620DD94FEA002343F000434D
:1028200010F0004F23FA02F018BF404270474FF0FB
:102830000000704712F1610F01D1420205D110F082
:10284000004008BF6FF0004070474FF00000704735
:102850005822024B4FF0FF301A607047B40000203E
:102860005822024B4FF0FF301A607047B40000202E
:102870005822024B00201A60704700BFB4000020AD
:102880005822024B4FF0FF301A607047B40000200E
:102890005822024B4FF0FF301A607047B4000020FE
:1028A000044A05491368002B08BF0B461844106002
:1028B00018467047B8000020701500205822024BBF
:1028C0004FF0FF301A607047B4000020334A34499B
:1028D00092F800C001F80C0008780CF10103DBB29B
:1028E0005528137002D00023137070470A2B0BD9A0
:1028F00010B44B78503B092B0DD8DFE803F01017CC
:102900001E252C333A4148067047264CD1F8020068
:10291000254B616803C30023137010BC7047214C22
:10292000D1F80200214B616803C3F4E71D4CD1F8D4
:1029300002001F4B616803C3EDE71A4CD1F8020097
:102940001C4B616803C3E6E7164CD1F802001A4B32
:10295000616803C3DFE7134CD1F80200174B6168CD
:1029600003C3D8E70F4CD1F80200154B616803C3CD
:10297000D1E70C4CD1F80200124B616803C3CAE7DF
:10298000084CD1F80200104B616803C3C3E7054C43
:10299000D1F802000D4B616803C3BCE706020020BA
:1029A0000C0100200E010020FC000020040100208A
:1029B000BC000020DC000020C4000020EC0000204F
:1029C000CC000020F4000020E4000020D40000200F
:1029D00070B50A21482001F08BF94FF4612000F016
:1029E000B3FD4FF47A7001F0C5F94FF47A7001F03D
:1029F000C1F900F0A9FE00F065FD01F051FB0021D6
:102A00004FF4616001F062FB1A4C01F041FB01F0F0
:102A100043FC01F07FFC00F059FA05E000F07CFD7A
:102A20004FF47A7001F0A6F901F0FEF80646207026
:102A30000028F3D100F068FD4FF47A7001F09AF9A4
:102A40000D4D2B78012B11D000F09CFB0028F8D005
:102A500000F08EFB044600F08FFB0146204600F09C
:102A6000ABFB00F095FB2B78012BEDD12E7000F025
:102A700039F8E9E7640000208002002070B50546BF
:102A80000C46154E304601F039F8B6F90610134AD7
:102A90002980B6F90810124B6980B6F90A10A9808E
:102AA000B6F90C102180B6F90E106180B6F910103D
:102AB000A180B5F90010B5F902001180B5F9041034
:102AC00050809180B4F90000B4F90210B4F90420E8
:102AD000188059809A8070BD1802002008020020DA
:102AE0001002002070B501F01BFC284BD3E9002434
:102AF00052EA040526D0801A4FF00002244D61EB03
:102B00000401854272EB01011CD200200021214CFE
:102B1000C3E900012260204C226000241F4A204BA0
:102B20002146012014601C6001F048FB2146022070
:102B300001F044FB1B4800F0EFF9BDE870401A4873
:102B400000F0EAB9134B1A68134B19680AB9002947
:102B5000E3D0144B154C1A841548226800685A8437
:102B60000E4C114B0E4D134E1984B26829465884F1
:102B7000204600F00FFA2D682168012001F01EFBAD
:102B80002946BDE87040022001F018BB3802002041
:102B900080841E004C0200206C0200206002002095
:102BA0006402002090020020B402002048020020AD
:102BB00068020020840200202DE9F84F4A4C984614
:102BC000D4E9007C57EA0C0305460E4691467ED0B8
:102BD000C01B61EB0C01FFF709FC4449FFF700FD46
:102BE00007460220C4E9005601F02CFA022001F049
:102BF00019FA0446042001F025FA042001F012FA23
:102C000003463B493B4A0D680C60641B1568384617
:102C100013605D1BFFF770F80F4606462046FFF76E
:102C2000D7FBFFF769F82CA3D3E90023FFF7BCF823
:102C30000022314BFFF7B8F829A3D3E90023FFF7AF
:102C4000DDF932463B46FFF7D9F90A4601462846E8
:102C50000C461546294BDFF8A8B0C3E90045FFF73D
:102C6000B7FBFFF749F81CA3D3E90023FFF79CF853
:102C70000022214BFFF798F819A3D3E90023FFF7AF
:102C8000BDF932463B46FFF7B9F906460F461D4BE4
:102C90002946C3E900672046FFF798FA3946CBF882
:102CA00000003046FFF792FADFF85CA02946CAF828
:102CB00000002046FFF78AFA034639463046A9F855
:102CC0000030FFF783FAA8F80000BDE8F88F0F4F37
:102CD00087E700BFAFF30080F701486DE25C354045
:102CE000000000000048A240400200200024744977
:102CF00050020020700200200000244058020020F2
:102D00004802002078020020680200200AD7233CF5
:102D1000F8B50D461C460746164601F001FBB5F511
:102D2000AA6F0A4BA8BF4FF4AA65B4F5AA6FA8BF53
:102D30004FF4AA64C3E9000107B96D42044B1D605A
:102D400006B96442034B1C60F8BD00BF3802002086
:102D50004C0200206C02002010B50121084803F04D
:102D60003DFD00B910BD0121064A074C1368044817
:102D70000B4413602170BDE8104003F03BBD00BF61
:102D8000002C01406C15002080020020F0B587B0B7
:102D90006C460C9F8DF80C2012128DF80D20B0F9A6
:102DA00004200D9E4FEA172E8DF810708DF811E05B
:102DB0008DF804204FEA174E12123F0E8DF8137053
:102DC0008DF80520370AB1F900208DF814608DF8D0
:102DD0001570370C360E8DF817608DF80E30B0F97F
:102DE00002601B128DF8062012128DF80F308DF83C
:102DF0000720B0F90030B1F90420B1F902008DF8D4
:102E0000026036128DF803608DF80800DEB28DF88E
:102E10000A201B12001212128DF816708DF8013064
:102E20008DF812E08DF800608DF80900A4460025A9
:102E300033468DF80B200DF1170701E01CF8013F18
:102E40002B44BC45DDB2F9D1552000F0D7FB102052
:102E500000F0D4FB182000F0D1FB01E014F8016F62
:102E6000304600F0CBFBBC42F8D1284600F0C6FB50
:102E7000BB2007B0BDE8F04000F0C0BB30B54FF458
:102E8000004089B003F02CF808B909B030BD01F05A
:102E900047FA05460C4604A806A9FFF7EFFD2846A9
:102EA00021460DF10E0303AAFFF786FEBDF90E3091
:102EB000BDF90C2004A806A9CDE90054FFF766FF70
:102EC0004FF4004003F01AF809B030BD0120F0B40F
:102ED000002240F2333702264FF480654FF461142C
:102EE0000B490C4B087718770F611F614E615E61CB
:102EF0008D619D61CC60DC60C1E90022F0BCC3E95A
:102F00000022CA830A628A60DA831A629A60704772
:102F100090020020B40200200023C0E90033836047
:102F2000704700BF2DE9F0411446984657680E1AC5
:102F300023692068F21B03FB02006369D21B03FBB9
:102F40000600A368D8F800501A44A36903FB0200E6
:102F5000FFF73EFA2946FFF785F9D8F80410FFF786
:102F60008BFA2946FFF780F9FFF74CFC0546FFF77F
:102F70002FFAE368C8F800009D422560A8BF1D46EF
:102F80005B42AB42B8BF2B46C4E901679812BDE86B
:102F9000F08100BF00232DE9F0472C4CDFF8B0A0F2
:102FA000227FD0F80090012A0E6880460F46CAF8AA
:102FB000003029D0C4E90033E383A3600223254D08
:102FC00023772B7F012B30D000230222C5E9003369
:102FD0002A77EB83AB60B4F91E301F4A4B4493420F
:102FE000B8BF13469642B8BF1646B3F5616FA8BF87
:102FF0004FF46163B6F5616FA8BF4FF46166C8F81E
:1030000000303E60BDE8F087144B2246B4F9221030
:10301000B4F92000FFF786FFDAF800300D4D0344C5
:103020005B42E3832B7F012BCED12A460B4BB5F9B4
:103030002210B5F92000BAF800A0FFF773FFAAEB41
:10304000000000B2E8830644C5E700BF90020020FC
:10305000D8020020B4020020F0F1FFFF740000202D
:10306000F8B50C461B4907461546FFF7C1FB00287B
:103070002ED120461749FFF7BBFB48BB2846154910
:10308000FFF7B6FB064618BB134B4FF089411F6094
:10309000124B38461C60124B124F1D60FFF7ECF9C3
:1030A000FFF7B0FB03464FF089413B612046FFF735
:1030B000E3F9FFF7A7FB03464FF089417B61284600
:1030C000FFF7DAF9FFF79EFBC7E90066BE60B8615B
:1030D000F8BD00BF00002041700000206C000020FF
:1030E0006800002090020020F8B50C461B490746F6
:1030F0001546FFF77DFB00282ED120461749FFF724
:1031000077FB48BB28461549FFF772FB064618BBFC
:10311000134B4FF089411F60124B38461C60124B15
:10312000124F1D60FFF7A8F9FFF76CFB03464FF045
:1031300089413B612046FFF79FF9FFF763FB034698
:103140004FF089417B612846FFF796F9FFF75AFB5C
:10315000C7E90066BE60B861F8BD00BF000020414D
:10316000700000206C00002068000020B4020020E5
:1031700000487047E0020020014B1878704700BFFC
:10318000DD020020014B1878704700BFDC020020F0
:1031900010B5064C22781AB100210548FDF710F849
:1031A0000023044A2370137010BD00BFDD0200200D
:1031B000E0020020DC02002070B50446881E0328CF
:1031C00040F381800323002214F803C00133DBB2F3
:1031D00098426244F8DCD2B2214411F8023C934296
:1031E00002D12378552B00D070BD6378013B082BAA
:1031F000FAD801A252F823F0B3320008E9310008EE
:10320000E9310008E9310008E9310008E931000836
:1032100095320008593200081D320008B4F8070042
:10322000FFF7D2F82C49FFF7DBF90546B4F80500A3
:10323000FFF7CAF82849FFF7D3F90346B4F80300AB
:103240001C46FFF7C1F82449FFF7CAF92A46214670
:10325000BDE87040FFF748BFB4F80700FFF7B4F8C7
:103260001D49FFF7BDF90546B4F80500FFF7ACF8B6
:103270001949FFF7B5F90346B4F803001C46FFF7F8
:10328000A3F81549FFF7ACF92A462146BDE870407E
:10329000FFF7E6BEE3781BB12379D3B100F034F930
:1032A0006379002BA0D0A3797BB1BDE8704000F01A
:1032B0003BB9B4F90730A279B4F90410E078BDE85D
:1032C0007040FFF725BD002286E7BDE8704000F0A2
:1032D00033B900F021F9E3E700007A44202330B548
:1032E000FC2587B08DF80530030A8DF80730030CF4
:1032F0008DF808300B0A8DF806008DF80A10000EC4
:103300008DF80B300B0C090E8DF804508DF80C3035
:103310008DF809008DF80D1001F002F84FEA102E1B
:103320008DF80FE08DF80E004FEA104E000E8DF86C
:103330001100080A01AC8DF812108DF81300080C6A
:10334000090E2A4623464FF0000C0DF115058DF8A5
:1033500010E08DF814008DF8151001E013F8012F1E
:10336000AB4282EA0C0CF9D1DF23FC208DF816C0A9
:1033700004F113058DF8173001E014F8010F00F087
:103380003DF9AC42F9D107B030BD00BF38B5474C6C
:103390002378042B06D8DFE803F019031C0F120072
:1033A00020286BD000232370414B1A78032A05D8BC
:1033B000DFE802F0434A351B0423237038BDDF28C1
:1033C0006DD0FC28EED10123237038BDFC28EBD151
:1033D000F9E7012860D00021354B21701A78032AC3
:1033E000ECD8DFE802F02A331C02324C3249227852
:1033F0008854324801320078D2B282422270DDD342
:10340000084410F8012CBB2A4FF0000239D0C1E962
:1034100000228A602270C1F80B201A7038BD421D4C
:10342000D2B226490E2A0A701FD90022214C224806
:1034300022701A7002800A7038BD552827D00022E9
:103440001D491A700A7038BD012807D0C21F012A11
:1034500004D9002218491A700A8038BD0222164C7D
:10346000144960701A700A7038BD03241149124D56
:103470000A781C70A85401320A7038BD02232370E8
:1034800038BD01200E49227008701A7038BD012223
:10349000094908701A7038BD0323237038BD00F045
:1034A0003FFFFFF71BFF0023237038BDF102002010
:1034B000EF020020F0020020E0020020DD020020E8
:1034C000DC02002000B5012183B0112002F064FB72
:1034D0000121092002F060FB4FF4005241F2030386
:1034E00001A90748ADF80420ADF8063002F086FACD
:1034F000044801A902F082FA03B05DF804FB00BFA2
:1035000000100140000C01404FF40051014802F04E
:10351000D9BA00BF001001404FF40051014802F039
:10352000CFBA00BF001001404FF40051014802F033
:10353000C7BA00BF000C01404FF40051014802F02F
:10354000C1BA00BF000C0140F0B5012187B00646AA
:1035500044F2040002F020FB4FF40073ADF8003099
:1035600041F60303234F69463846ADF8023002F0B6
:1035700045FA4FF48063ADF80030042369463846BD
:1035800000258DF8033002F039FA4FF440231A4C2D
:1035900002A920460493CDE90265ADF8145002F06B
:1035A0002BFB2A46204640F2277102F08FFB0122B6
:1035B000204640F2255102F089FB2046402102F0CE
:1035C000A7FB0121204602F073FB4FF4A06002F03C
:1035D000D5F901232521032201A88DF805308DF8A6
:1035E00004108DF806208DF8073002F0D1F907B0ED
:1035F000F0BD00BF0008014000380140844610B40F
:10360000064A074C13780748591C117004F803C088
:10361000012240F2277110BC02F058BBF5030020D4
:10362000F40200200038014038B540F227711B48F1
:1036300002F072FB30B940F22551184802F06CFBE1
:10364000D0B938BD164C17492378174D5A1CC95CA0
:103650001248227002F054FB22782B789A4213D041
:1036600040F227710D4802F079FB40F225510B48DA
:1036700002F052FB0028E4D0084802F045FBBDE808
:103680003840C0B2FFF782BE002240F227710348E3
:1036900002F01CFB002323702B70E1E7003801408F
:1036A000F4030020F4020020F503002038B5224C7A
:1036B00040F22771204602F02FFBC8B11F4D204A6F
:1036C0002B782046D15C01332B7002F019FB40F2BD
:1036D0002771204602F042FB1A4B2A781B789A4247
:1036E0001DD0BDE838404FF45871134802F036BB86
:1036F00040F22551204602F00FFB0028F1D0A088AF
:10370000C0B2FFF7E3F8204640F2255102F026FB55
:10371000BDE838404FF45871074802F01FBB2046FF
:1037200040F22771002202F0D1FABDE838404FF490
:103730005871014802F012BB00480040F804002014
:10374000F8030020F904002030B5012187B04FF4C0
:10375000017002F021FA4FF4004002F0CBF900248E
:10376000102369461748ADF800308DF8034002F089
:1037700045F9154802F0FAFA01254FF46023124882
:1037800001A903930194ADF8084004948DF81450F6
:1037900002F022FB0C48294602F044FB0A4802F0E2
:1037A0004BFB094802F04EFB0028FAD1064802F014
:1037B0004DFB054C204602F04FFB0028FAD107B024
:1037C00030BD00BF000801400024014030B5012198
:1037D00085B0042002F0E0F94FF400444823694624
:1037E00014488DF80330ADF8004002F007F90F21BE
:1037F000002002F069F9204602F080FB0125282113
:103800000222032301A88DF804108DF805208DF8FD
:1038100006308DF8075002F0BBF84FF4006302A8A1
:1038200002948DF80E50ADF80C3002F019FB05B083
:1038300030BD00BF0008014010B5012186B04FF433
:10384000800002F0B5F90121082002F0A5F94FF43B
:10385000406241F60343104C01A91048ADF8042022
:10386000ADF8063002F0CAF8204602F0C7FF4FF468
:1038700080430B480B490C4ACDE90201204602A9BE
:103880000492ADF8143002F0D7FF0121204603F076
:1038900043F806B010BD00BF00580040000C0140C6
:1038A000801A06000000FFBF090000042DE9F04166
:1038B000804626480E4601214FF47A740546244F6F
:1038C00003F038F801E0013C05D03946284603F002
:1038D0006DF80128F7D10022D0211C4803F05AF8D6
:1038E0004FF47A741B4F194D01E0013C05D0394665
:1038F000284603F05BF80128F7D14146134803F04E
:1039000043F84FF47A74144F104D01E0013C05D098
:103910003946284603F04AF80128F7D131460B48CA
:1039200003F032F84FF47A740C4E084D01E0013C7C
:1039300005D03146284603F039F80128F7D1012196
:10394000BDE8F041014803F003B800BF0058004053
:1039500001000300820007008000070084000700C8
:10396000F8B507463A4801214FF47A740546394EB6
:1039700002F0E0FF01E0013C05D03146284603F0AB
:1039800015F80128F7D10022D021314803F002F8C0
:103990004FF47A74304E2E4D01E0013C05D0314693
:1039A000284603F003F80128F7D13946284802F0E9
:1039B000EBFF4FF47A74294E254D01E0013C05D010
:1039C0003146284602F0F2FF0128F7D101212048B4
:1039D00002F0B0FF4FF47A741E4E1D4D01E0013C21
:1039E00005D03146284602F0E1FF0128F7D1012237
:1039F000D021174802F0CEFF4FF47A74184E144DC0
:103A000001E0013C05D03146284602F0CFFF0128F5
:103A1000F7D100210E4802F0A9FF01210C4802F065
:103A200097FF4FF47A740F4E094D01E0013C05D029
:103A30003146284602F0BAFF0128F7D1044802F0C7
:103A4000A5FF04460121024802F090FF2046F8BD80
:103A500000580040010003008200070084000700B6
:103A600002000300400003000C4B00B5D0F800C07A
:103A7000416882681B68D0F80CE0C3F800C0596048
:103A80009A60C3F80CE0D0F810C041698269C3F8AD
:103A900010C059619A615DF804FB00BFFC0400206E
:103AA00093B1F8B500240E4617461D46A4463019BA
:103AB000013417F80C10E4B2C0B2FFF7F7FEAC42C5
:103AC000A446F4D30020F8BD00207047A3B12DE92F
:103AD000F04100240F4690461E4625463819C0B2D4
:103AE000FFF73EFF0134E4B2B44208F80500254672
:103AF000F4D30020BDE8F08100207047034620B1D8
:103B0000034A0448136000F0A3BF4FF0FF30704732
:103B1000FC0400200005002030B585B001A936481E
:103B200001F084FA0199044602AA334801F0EAFA46
:103B3000044351D19DF90830012B1ED02F4C304D3C
:103B40009DF909102F4801290CBF29462146FCF791
:103B50009FFB9DF90A102C4801290CBF29462146DC
:103B6000FCF796FB9DF90B10284801290CBF29464C
:103B70002146FCF78DFB4FF0FF349DF90C30012BF3
:103B800023D01E4C1E4D9DF90D10214801290CBF5C
:103B900029462146FCF77CFB9DF90E101D480129A2
:103BA0000CBF29462146FCF773FB9DF90F101A48FC
:103BB00001290CBF29462146FCF76AFB9DF80C3011
:103BC0009B0758BF4FF0FF340DD4144D20462B688F
:103BD00001332B6005B030BD104D224629681048D6
:103BE000FCF756FBF2E70D4D0E482968FCF750FB39
:103BF0004FF0FF34EAE700BF00050020946A000898
:103C0000906A0008D06A0008E06A0008F06A0008BC
:103C1000006B0008106B0008206B0008581500208E
:103C2000986A0008306B000830B5002489B08DF820
:103C30000740FFF701FEFFF7C9FD4FF480632849F5
:103C4000284A294DCDE903122846224602A9CDE98A
:103C500005330794029401F093F810B140B209B013
:103C600030BD224B28460DF107012B6200F028FCE5
:103C700098BB9DF80730672B2CD1FFF74DFF04460A
:103C800060B10325FFF740FCC82000F073F8FFF790
:103C900043FCC82000F06EF8013DF3D160211248CA
:103CA00000F0D2FC0921104800F0AEFC0E4800F0F4
:103CB0000FFC00210C4800F0ADFD09210A4800F07E
:103CC00089FD094800F0E0FC642000F053F860B280
:103CD00009B030BD6FF00200C1E76FF00100BEE730
:103CE000CD3A0008A13A000800050020693A000812
:103CF0000346F0B503254FF0E022002403FB01F159
:103D0000C1EB411CEB4001EB8C01104F9461516100
:103D10001561C3EB43123B700D4E03EB820383B07E
:103D2000AB404FF4C060338001F028FEFF22012336
:103D300001A88DF805508DF806408DF804208DF807
:103D4000073001F025FE03B0F0BD00BF5E15002076
:103D50005C1500200121054A054B11701A781AB133
:103D60001A78013AD2B21A70704700BF601500206D
:103D70005F1500204FF0E02C234A244B128800B539
:103D800002FB00F0DCF81820DCF81410B0FBF1F1B5
:103D9000C9B21970DCF81410B0FBF1FE01FB1E0073
:103DA000824213D9101A1A78002AFCD109284FF040
:103DB000E02204D893690A2BFCD85DF804FB9369D0
:103DC0008342FAD993698342F9D8F6E71978013129
:103DD000C9B21970DCF814100A44101A1A78002AB3
:103DE000FCD109284FF0E02206D893690A2BE4D9C8
:103DF00093690A2BF9D8E0E793698342DDD9936987
:103E00008342F9D8D9E700BF5C1500205F15002078
:103E10004FF0E02C00B5234A234B127802FB00F050
:103E2000DCF81820DCF81410B0FBF1F1C9B21970FD
:103E3000DCF81410B0FBF1FE01FB1E00824213D926
:103E4000101A1A78002AFCD109284FF0E02204D871
:103E500093690A2BFCD85DF804FB93698342FAD975
:103E600093698342F9D8F6E719780131C9B219701C
:103E7000DCF814100A44101A1A78002AFCD1092818
:103E80004FF0E02206D893690A2BE4D993690A2BF4
:103E9000F9D8E0E793698342DDD993698342F9D881
:103EA000D9E700BF5E1500205F150020F0B50121A5
:103EB00089B0022001F07CFE04260121042001F0DB
:103EC0006BFE4023264F0DEB06013846ADF804305B
:103ED0008DF8076001F092FD3046012101F05CFE93
:103EE00080230DEB06013846ADF804308DF80760ED
:103EF00001F084FD02A802F0DDFB00254FF6FF7300
:103F0000184C02A92046ADF80C30ADF80850ADF8B9
:103F10000E50ADF80A5002F09DF92A462B460321B7
:103F2000204602F0FBFB05A802F0D8FB0A2320463E
:103F300005A9ADF81C3002F0FDFA2046012102F07F
:103F400049FC01222046114602F0DEFB47F6FF73D2
:103F500001212046A38402F0C9FB09B0F0BD00BFD7
:103F60000008014000040040F0B5012189B00420A0
:103F700001F01EFE04270121082001F00DFE402360
:103F8000264E0DEB07013046ADF804308DF8077072
:103F900001F034FD0121082001F0FEFD80230DEB2E
:103FA00007013046ADF804308DF8077001F026FDAA
:103FB00002A802F07FFB00254FF6FF73184C02A900
:103FC0002046ADF80C30ADF80850ADF80E50ADF805
:103FD0000A5002F03FF92A462B460321204602F000
:103FE0009DFB05A802F07AFB0A23204605A9ADF83F
:103FF0001C3002F09FFA2046012102F0EBFB012267
:104000002046114602F080FB47F6FF73012120464F
:10401000A38402F06BFB09B0F0BD00BF000C0140AF
:1040200000080040022805D0042806BF034B18688A
:1040300000207047024B1868704700BF68150020C9
:104040006415002002280ED004280BD147F6FF7318
:104050000B490C4A888C8B8411681B1A1BB20B44C9
:1040600013607047704747F6FF73074A0749908C03
:1040700093840A681B1A1BB2D31A0B60704700BFE7
:10408000000800406815002000040040641500206E
:1040900008B5FFF70BFFBDE80840FFF765BF00BF9D
:1040A00000B5012183B0042001F076FD0F2241F616
:1040B0000303054801A9ADF80420ADF8063001F06E
:1040C0009DFC03B05DF804FB000801402DE9F043BE
:1040D00089460121064600250C464FF0600802275C
:1040E00089B0084601F064FD4FF0804001F098FF70
:1040F000013E01A94FF08040ADF80A50ADF80650DE
:10410000ADF80490ADF8086002F0A4F804A802F03D
:10411000DBFA04A94FF08040ADF81080ADF81240F2
:10412000ADF81650ADF8187002F0EAF808214FF01B
:10413000804002F029FB04A94FF08040ADF81080C8
:10414000ADF81240ADF81650ADF8187002F026F92F
:1041500008214FF0804002F01FFB04A94FF080407F
:10416000ADF81080ADF81240ADF81650ADF81870EB
:1041700002F05CF908214FF0804002F017FB04A91F
:104180004FF08040ADF81080ADF81240ADF81650F9
:10419000ADF8187002F092F94FF08040082102F05B
:1041A0000DFB21464FF0804002F0E0FA21464FF02F
:1041B000804002F09BFA09B0BDE8F08338B5344B7B
:1041C0009942B8BF1946B1F5616FA8BF4FF461615C
:1041D00001281BD0022818D10846FEF7F9F8002163
:1041E0000446FEF7FBFA034648B32046FDF784FD7C
:1041F0000022284BFDF702FFFEF710F84FF0804336
:10420000002280B29887A3F8402038BD0846FEF708
:10421000DFF800210546FEF7E1FA044620B300234B
:104220004FF080442846A386FDF766FD0022194B17
:10423000FDF7E4FEFDF7F2FF80B2208738BD4FF0B6
:1042400080452046AB87FEF7DDFA0028B8BF404224
:10425000FDF740FD00220F4BFDF7D0FEFDF7DEFF1E
:1042600080B2A5F8400038BD2846FEF7CBFA0028FA
:10427000B8BF4042FDF72EFD064B0022FDF7BEFE03
:10428000FDF7CCFF4FF0804380B298861C8738BD85
:10429000F0F1FFFF0000F83F70B5012184B04FF44A
:1042A000006001F079FC00254723012642F20F72DD
:1042B000174C01A92046ADF80430ADF80820ADF840
:1042C0000A50ADF806508DF80C5001F0C3FF32468D
:1042D0003146204602F018FA4FF4A06001F04EFB80
:1042E00019220223032168468DF800208DF8013041
:1042F0008DF802108DF8036001F04AFB314620462C
:1043000002F0F4F92946204602F062FA04B070BDCA
:10431000002C01400022014B1A6070476C150020F0
:104320000D4910B40D4C8A8C2368888C92B280B2EF
:10433000824203D92268934207D01346002142F2F9
:104340000F7210BCE3FB020170478A8C92B2B2F587
:104350007A7FF3D20133F1E7002C01406C15002085
:10436000F0B5002583B001222E490DF10703064662
:104370008DF8075001F08AF90DF107030746012275
:104380003046294901F082F97369074363B3012B71
:1043900026D0022B42D18DF8075001224FF0011197
:1043A0000DF10703304601F071F9012204461F495F
:1043B0000DF10703304601F0BDF89DF807200546D2
:1043C00042F003028DF807203046012217490DF113
:1043D000070301F05BF92C433C43204303B0F0BDDD
:1043E00004238DF80730D8E70DF10703012230468A
:1043F0000F4901F09FF89DF80720054622F00C02B6
:104400008DF807203046012209490DF1070301F01C
:104410003DF9054345EA070003B0F0BD6FF00A001F
:10442000DCE700BF7C0001007900010035000100DD
:104430003600010030B5002483B00DF107030122DE
:104440001B4905468DF8074001F020F90DF10703DF
:10445000012204461749284601F018F94FF0100CC4
:104460008646012214490DF10703284644EA0E044A
:104470008DF807C001F00AF903464FF47A701C4327
:1044800001F0E0F92846FFF76BFF84460DF10703C2
:1044900001222846094944EA0C0401F04BF89DF832
:1044A00007302043102B18BF60F00B0003B030BD65
:1044B0007C00010079000100020001003A000100C7
:1044C0000B460122014901F035B800BF750001001B
:1044D000F0B583B00DF1050301224749044601F010
:1044E00029F89DF80530054603F00307022F26D072
:1044F000012241490DF10503204601F01BF89DF80A
:104500000520064622F0030242F003020DF10503E6
:104510008DF8052020460122374901F0B7F80346FF
:10452000C8201E43354301F08DF92FB904F580539F
:1045300093F84730002B56D1284603B0F0BD1B0737
:1045400031D401222D490DF10603204600F0F2FF7F
:104550009DF8063045EA000603F00F03053B092BE2
:1045600098BF274A244998BF52F8237020464FF03D
:1045700001020DF1070388BF224F00F0DBFF9DF819
:104580000720054662F07F020DF107038DF8072032
:1045900020460122184901F079F803463543384690
:1045A0001D4301F04FF90DF1050301222046124988
:1045B00000F0C0FF9DF805200F4922F0030242F0F1
:1045C00003020DF105038DF8052006460122204661
:1045D00001F05CF82E430546C820354301F032F95E
:1045E000284603B0F0BD01F02FF904F58254C4E968
:1045F0000401284603B0F0BD1F00010021000100A6
:10460000546B000800C40900F0B50E4F83B00DF1E3
:1046100007030C4601223946064600F08BFF9DF841
:104620000720054622F00F02144339463046012286
:104630000DF107038DF8074001F028F8284303B077
:10464000F0BD00BF21000100F0B50E4F83B00DF1A9
:1046500007030C4601223946064600F06BFF9DF821
:104660000720054622F060021443394630460122F5
:104670000DF107038DF8074001F008F8284303B057
:10468000F0BD00BF210001002DE9F04182B0012200
:104690000DF105034B49044600F04CFF9DF8053031
:1046A000064603F00302022A03F00C0726D001227B
:1046B00044490DF10503204600F03CFF9DF805201C
:1046C000054622F00C0242F00C020DF105038DF8B4
:1046D0000520204601223B4900F0D8FF0346354320
:1046E000C8201D4301F0AEF827B904F5805393F8B4
:1046F000473043BB284602B0BDE8F0811B072CD5EC
:104700000DF10503012220462E4900F013FF8446D7
:104710009DF805202B4922F00C0242F00C020DF10D
:1047200005038DF8052020460122644600F0AEFF07
:1047300005462C43C82044EA060501F083F82846C4
:1047400002B0BDE8F08101F07FF804F58254C4E9BD
:104750000201284602B0BDE8F08101220DF10603F6
:104760002046194900F0E6FE9DF8063046EA0005AD
:1047700003F00F03053B092B98BF144A204698BF4E
:1047800052F823800F490DF107034FF0010288BF53
:10479000DFF83C8000F0CEFE9DF80720064662F070
:1047A0007F020DF107038DF80720204601220549FD
:1047B00000F06CFF03463543404645EA030601F02E
:1047C00041F874E71F00010021000100546B00084C
:1047D00000C40900F0B50E4F83B00DF107030C467D
:1047E00001223946064600F0A5FE9DF80720054641
:1047F00022F00F0214433946304601220DF107031F
:104800008DF8074000F042FF284303B0F0BD00BF21
:1048100020000100F0B50E4F83B00DF107030C46E8
:1048200001223946064600F085FE9DF80720054620
:1048300022F0600214433946304601220DF107038D
:104840008DF8074000F022FF284303B0F0BD00BF01
:104850002000010030B583B0054600F071FE0DF177
:104860000703012203210446284600F063FE844624
:104870009DF80730012223F070038DF807300321E3
:104880000DF10703284644EA0C0400F0FFFE8446BD
:104890000DF1070301220021284644EA0C0400F030
:1048A00049FE84469DF80720002122F002020DF106
:1048B00007038DF807202846012244EA0C0400F083
:1048C000E5FE034628461C4300F020FD204303B0CC
:1048D00030BD00BF70B50C4682B00DF10703012258
:1048E0002249064600F026FE9DF807200DF1070339
:1048F000C2F380112170C2F3C0016170C2F3800164
:10490000C2F34002A170E270054601223046184908
:1049100000F010FE012284469DF807103046C1F3D6
:10492000C006267101EA02066671C1F34006C1F3B2
:1049300080010DF10703E171A6712F2145EA0C05F5
:1049400000F0F8FD9DF807302843DA092272C3F31E
:1049500080126272C3F34012A272C3F30012C3F357
:10496000C003E272237302B070BD00BF2B000100D0
:104970002C000100F0B50C4683B0022201AB334994
:10498000074600F0D7FD9DF904302278054623F054
:104990004E030AB143F0400362780AB143F00803C2
:1049A000A2780AB143F00403E2780AB143F00203AB
:1049B00022798DF804309DF905306179002A23F0C1
:1049C0000F0314BF08220022002918BF43F001037F
:1049D0001343A2790AB143F00203E2790AB143F02A
:1049E0000403022219498DF80530384601AB00F066
:1049F0004DFE2F21064601AB0122384600F09AFDFC
:104A00009DF80410237A0643354301F007010BB1EA
:104A100061F07F01637A0BB141F04001A37A0BB1E1
:104A200041F02001E37A0BB141F01001237B0BB17F
:104A300041F008018DF80410012238462F2101AB06
:104A400000F024FE284303B0F0BD00BF2B0001009E
:104A500070B58EB0012238490DF10703054600F00C
:104A600069FD044618B99DF80730DB0702D42046DB
:104A70000EB070BD02AB02222846304900F05AFD4C
:104A800005F5805696F845300446102B3BD0BDF90D
:104A90000810062203ABADF82E102846284900F076
:104AA00049FD96F84530BDF80C20102B44EA00046F
:104AB000BDF80E3035D0BDF91010ADF82220ADF89C
:104AC000243005ABADF8261006221E49284600F01A
:104AD00031FD96F84530BDF81410102B44EA00045F
:104AE000BDF8163013D0BDF91820ADF82810ADF878
:104AF0002A302B6AADF82C20002BB8D007A8984795
:104B000020460EB070BDBDF80810C9BAC1E7BDF8A7
:104B1000182049BA5BBAADF82810ADF82A30D2BADD
:104B2000E7E7BDF8101052BA5BBAADF82220ADF835
:104B30002430C9BAC5E700BF3900010009000100EF
:104B40000B00010011000100042370B582B004467F
:104B50008DF8073000F0F4FC0DF107030646012242
:104B60002046124900F092FD03460A201E4300F041
:104B700069FE6EB90D4D07E00122294620460DF170
:104B8000070300F0D7FC48B99DF807305B07F3D462
:104B9000204600F0BBFB304302B070BD0646204605
:104BA00000F0B4FB304302B070BD00BF0200010052
:104BB000F0B500260F4600F5805387B083F8471004
:104BC0000546CDE9026604968DF8146000F0B8FC45
:104BD000002F00F08880012F7DD13A460DF10703A8
:104BE0002846644900F0A6FC9DF807303A4623F0B9
:104BF000600343F040038DF8073004460DF10703CE
:104C000028465C4900F042FD3A460DF107035A4937
:104C10000443284600F08EFC9DF807303A4623F006
:104C2000030343F002038DF8073053490DF10703E6
:104C30000443284600F02AFD3A4631460DF10703A9
:104C40000443284600F076FC9DF807303A4623F0EE
:104C5000010343F0010331468DF8073004430DF1A1
:104C60000703284600F012FD3A4639460DF10703C6
:104C70000443284600F05EFC9DF807303A4623F0D6
:104C80000F0343F0270339468DF8073004430DF135
:104C90000703284600F0FAFC3A460DF107033749AE
:104CA000044328468DF8077000F0F0FC034602A983
:104CB00028461C43FFF70EFE034602A928461C4364
:104CC0008DF80960FFF756FE0443284600F01EFBEE
:104CD000204307B0F0BD28464FF0FF3400F016FB2C
:104CE000204307B0F0BD0DF10703012228462249F9
:104CF00000F020FC9DF80730044623F0010343F048
:104D000001038DF8073001220DF1070328461A49E7
:104D100000F0BCFC012201460DF1070328460C43BC
:104D2000114600F007FC01229DF80710064621F00D
:104D3000070141F004010DF107038DF80710284623
:104D4000114600F0A3FC034602A9284634431C4345
:104D5000FFF7C0FD0123024602A9284614438DF83F
:104D60000930FFF707FE0443284600F0CFFA20433E
:104D700007B0F0BD35000100280001002900010046
:104D80002DE9F04F0D4617468BB041F25802002135
:104D90000446FBF715FA002D00F0ED806B68002B40
:104DA00000F0E980AB68002B00F0E5800FCD2646CF
:104DB0000FC695E8030086E8030040F6B83000F01F
:104DC00041FD0023276223772046FFF7C9FA0546F5
:104DD0002046FFF72FFB0746204600F019FC3D4315
:104DE000074601222046654906AB2F4300F0A2FB8F
:104DF000002800F0B7804FF0000807432046012646
:104E0000CDE90688CDF820808DF82480FFF722FDBB
:104E10003246414605460DF11703204600F08AFB55
:104E200084469DF81730324623F0080343F0080308
:104E3000414620468DF817300DF11703CDF808C014
:104E400000F024FC8446324620464D490DF11703FC
:104E5000CDF80CC000F06EFB84469DF8173032464A
:104E600023F0020343F00203204645498DF8173032
:104E70000DF11703CDF800C000F008FC844632465F
:104E800020463F490DF11703CDF804C000F052FB56
:104E90009DF81730324623F00103334383463849E7
:104EA00020468DF817300DF1170300F0EFFB06A92F
:104EB000824620468DF818808DF819808DF81B8069
:104EC0008DF81A608DF81C608DF81D608DF81E60DD
:104ED0008DF81F608DF820608DF821608DF82260BC
:104EE0008DF823608DF82460FFF744FD314681463C
:104EF0002046FFF75DFE32468046022120460DF136
:104F0000170300F017FB84469DF817103246314313
:104F100020460DF117038DF817100221664600F0A8
:104F2000B5FB029A45EA07031343039A04F582543A
:104F30001343009A1343019A134343EA0B0B4FF0B8
:104F4000FF3200234BEA0A0A4AEA090949EA08083B
:104F5000C4E90223C4E9042348EA060630430BB03F
:104F6000BDE8F08F9DF8182004F5805302F0100280
:104F700083F845203FE74FF0FF30F0E735000100B0
:104F80000600010000232DE9F04182B00646884664
:104F90008DF8073000F0D4FA234F0DF1070339469E
:104FA00001220446304600F0C5FA9DF8072008F0BB
:104FB000030822F0030242EA08028DF8072039466E
:104FC00001220DF107030443304600F05FFB044368
:104FD0004FF47A7041F2883500F034FC02E0013D74
:104FE0001BD374B90A2000F02DFC0DF10603012239
:104FF0003946304600F09EFA9DF8063004439B0780
:10500000EDD1304600F082F9002D40EA040008BFDF
:105010006FF0030002B0BDE8F081304600F076F991
:105020006FF00300F6E700BF250001000020C02359
:1050300008704B70704700BF30B583B0054600F074
:105040007FFA0DF1070301222B210446284600F0C8
:1050500071FA84469DF80730012223F00C0343F0D7
:105060000C038DF807302B210DF10703284644EA85
:105070000C0400F00BFB84460DF10703012242F6FD
:105080000601284644EA0C0400F054FA84469DF8D0
:105090000730012223F0020342F606018DF80730A3
:1050A00028460DF1070344EA0C0400F0EFFA03462A
:1050B00064201C4300F0C6FB0DF10703012242F6F9
:1050C0000601284600F036FA84469DF8072042F68D
:1050D000060122F0080242F008020DF107038DF8E4
:1050E00007202846012244EA0C0400F0CFFA0346C8
:1050F00014201C4300F0A6FB284600F007F92043CB
:1051000003B030BD2DE9F043002585B0ADF80410A3
:1051100003AB7C499046012206468DF80D508DF870
:105120000E5000F007FA9DF80C30012223F00F0317
:10513000744904468DF80C30304603AB00F0A6FAF3
:105140000443304600F0FCF9012104433046FFF7E8
:1051500019FF06F58053044383F844503046FFF7A7
:105160006BFF0DF10F0301221421044330469DF81B
:10517000047000F0DFF99DF80F3013F0C00F40F01D
:10518000BE808146012213210DF10F03304600F04D
:10519000D1F99DF80F20054622F07F021743132115
:1051A000012230460DF10F0347F03F078DF80F70D5
:1051B00000F06CFA054345EA09000122142104437A
:1051C00003AB304600F0B6F99DF80C309DF8052091
:1051D00003F03F0313430546012214218DF80C30E0
:1051E000304603AB00F052FA2C4304434FF47A707C
:1051F00000F028FB01220DF10E033046424900F079
:1052000099F99DF80E3040F2E73523F07F023E4FCA
:1052100004438DF80E2014E0ACB94FF47A7000F01E
:1052200011FB39460DF10E030122304600F082F9E0
:105230009DF80E30013D23F07F0104468DF80E10DD
:1052400058D01B06E8D50DF10D030122642130462C
:1052500000F070F99DF80D100DF10D03C1F341152B
:1052600088F80450C1F3400588F80550C1F3800563
:10527000C1F3C00188F8065088F8071005460122DE
:105280006321304600F056F99DF80D202C43C2F3FF
:10529000401188F80010C2F3400188F80110C2F3F1
:1052A0008001C2F3C00203AB88F8021088F8032023
:1052B000142101220443304600F03CF99DF80C20F3
:1052C000142102F03F02054603AB8DF80C20304656
:1052D000012200F0DBF903462C4330461C43FFF764
:1052E00033FC034630461C4300F010F8204305B061
:1052F000BDE8F0834FF0FF3005B0BDE8F0836FF0FC
:105300000B005AE71F0001003A00010070B582B09F
:1053100098B3067F0446012E13D00DF10703012236
:10532000194900F0A3F89DF8073013F0100F14BFCF
:1053300005464FF0FF35237F013B2377284602B017
:1053400070BD0DF1070332460F4900F08FF89DF84C
:105350000730054603F0EF038DF807302376236905
:1053600073B133461F212046A6680DF10702B047EE
:105370000028E0D065F00205DDE76FF00A05DDE703
:1053800060F00405D7E700BF1F000100F0B50B0A6D
:1053900083B08DF80730002862D00E4617460446C9
:1053A00000F0CEF89DF807300546002B38D1236970
:1053B0008DF80660002B47D001237D212046A6688A
:1053C0000DF10602B047002847D10A2000F03AFA52
:1053D000E368002B3BD001233A467E2120466668D5
:1053E000B047002836D10A2000F02CFA9DF807308B
:1053F0002BB92046FFF78AFF284303B0F0BD0022F7
:1054000023698DF8062073B301237C212046A6680A
:105410000DF10602B0470028EBD065F00205E8E781
:1054200023696BB101237C212046D4F808C00DF11B
:105430000702E04723690028BAD065F00205B7E704
:1054400060F004058DF8066065F00405BDE765F0C1
:105450000405C8E765F00205C5E765F00205B4E795
:105460006FF00A00C9E765F00405C2E72DE9F04FC7
:1054700083B017460193002A50D04FF0000A05462A
:105480000E461A465446DFF8A0B0DFF8A090DFF8C9
:10549000A0800BE0414508BF05F1180315D11B782A
:1054A0000134A742137002F101021DD0311965B118
:1054B00059451DD004D80029ECD105F11B03EEE7B6
:1054C000494502D105F11A03E9E7F30313D428464D
:1054D00089B20092FFF75AFF0134009AA7424AEAC4
:1054E000000A02F10102E1D1504603B0BDE8F08F9D
:1054F00005F11903D3E7019AC9B23B1B22447DB1E0
:10550000E868834288BF6AF0040AEDD828466C68D0
:10551000A0470028E8D06AF0020AE5E79246E3E7F0
:105520006AF00A0AE0E700BF200001002100010044
:105530001F00010008B1FFF799BF6FF00A00704724
:105540002DE9F04182B000285AD0037F0546A3B16F
:105550000DF1070301222C49FFF788FF9DF8073062
:1055600013F0100F14BF04464FF0FF342B7F0133AC
:105570002B77204602B0BDE8F08101220DF1070330
:105580002149FFF773FF9DF807302A6943F01003A4
:1055900004468DF807302B767AB301231F21284665
:1055A000AE680DF10702B04718BB002CE1D100F046
:1055B0004BF9DFF8588006460F4603E09DF80730A8
:1055C0001B07D3D401224FF4803128460DF1070385
:1055D000FFF74CFF04460028CBD100F035F9801BC3
:1055E00061EB0701804574EB0103E7D26FF0030420
:1055F000BFE76FF002031C43BBE76FF00403FAE759
:105600006FF00A04B5E700BF1F00010040420F0021
:10561000B0B338B5C368044600F118023BB30123A8
:1056200045681F21A847E368051E18BF6FF00205F3
:1056300004F119023BB3012320212046D4F804C011
:10564000E047D0B9E36804F11A02E3B10123212154
:105650002046D4F804C0E04760B90021204604F198
:105660001B02FFF793FE00232377284338BD6FF01A
:105670000405F2E765F00205EFE765F00205E1E7F2
:105680006FF00A00704765F00405E6E72DE9F04F7A
:1056900089B0CDE903210593002800F0C3800446BA
:1056A000002A00F0A7801E46002301F4803702EB99
:1056B000010801970D464746DFF87C91DFF87CA191
:1056C000DFF87CB102930DE05D4508BF04F11802DC
:1056D00001D133781370019B8BB10135BD4206F1C6
:1056E000010646D04D454AD004D8002DECD104F136
:1056F0001B02EEE75545EED104F11A02E9E7C5F3C6
:10570000072320468DF81F30FFF71AFF9DF81F3042
:105710008046002B4AD123698DF81E50002B78D08B
:1057200001237A212046D4F808C00DF11E02E0477B
:10573000002871D12369002B6BD0012332467B21D5
:105740002046D4F808C0E047002850D10A2000F0D5
:1057500079F89DF81F30ABB92046FFF7D7FD029BC3
:1057600040EA080001350343BD42029306F10106F9
:10577000B8D1019F4FBB029809B0BDE8F08F04F18A
:105780001902A6E700238DF81E302369002B46D0AE
:10579000012379212046D4F808C00DF11E02E0470C
:1057A000B0F1000818BF6FF00208D5E7236963B3B2
:1057B000012379212046D4F808C00DF11F02E047EB
:1057C0000028A8D068F00208A5E72369039A9DF88D
:1057D00010109A422AD82046039B059AA468A04735
:1057E0000028C8D0029B63F002030293C3E768F06D
:1057F0000208ABE7049B13F4803301D10293BAE7AC
:10580000039B9DF810100293E5E760F004088DF803
:105810001E5068F0040899E768F002088AE76FF004
:10582000040899E76FF00A030293A4E7029B63F070
:10583000040302939FE700BF200001002100010044
:105840001F000100FEF7E4BA42F21070024B002183
:105850001B6803FB00F070473402002010B40020E6
:105860004FF41F04394A3A4B116883B041F00101EB
:10587000116051680B405360136823F0847323F464
:1058800080331360136823F480231360536823F478
:10589000FE035360946000900190136843F48033DA
:1058A000136003E0009BB3F5A06F09D0136803F405
:1058B00000330193009B01330093019B002BF1D037
:1058C000224B1B6813F4003318BF01230193019B83
:1058D000012B06D04FF000621E4B9A6003B010BC43
:1058E00070471D4A194B116841F010011160116891
:1058F00021F003011160116841F0020111605A6842
:105900005A605A685A605A6842F480625A605A680B
:1059100022F47C125A605A6842F4E8125A601A68FB
:1059200042F080721A601A689201FCD55968074AE1
:1059300021F003015960596841F002015960536830
:1059400003F00C03082BFAD1C4E700BF001002409B
:105950000000FFF800ED00E000200240704700BFAB
:10596000FEE700BFFEE700BFFEE700BFFEE700BFA7
:10597000704700BF704700BF704700BF034B40F047
:10598000BF6040F40030D860704700BF00ED00E019
:10599000C37813B3174A30B5D1684FF0010EC9432D
:1059A0000F23827890F801C00078C1F3022100F043
:1059B0001F040EFA04F4CB40C1F1040E13400CFA9C
:1059C0000EFC0D4D43EA0C031B012A18DBB2400903
:1059D00082F8003345F8204030BD012103780648A5
:1059E0005A0903F01F03203201FA03F340F8223072
:1059F000704700BF00ED00E000E100E02DE9F0415C
:105A000091F803C01CF0100F18BF8B7809880CF0B8
:105A10000F0518BF1D43CBB21BB3002301264FF067
:105A20000F08046802E00133082B19D006FA03F2CC
:105A300032EA0107F7D14FEA830E08FA0EF724EA9B
:105A4000070405FA0EFEBCF1280F4EEA040432D01A
:105A5000BCF1480F03F1010308BF0261082BE5D137
:105A60000460FF2925D9002301264FF00F08446860
:105A700002E00133082B1BD003F1080206FA02F200
:105A800032EA0107F5D14FEA830E08FA0EF724EA4D
:105A9000070405FA0EFEBCF1280F4EEA04040CD0F0
:105AA000BCF1480F03F1010308BF0261082BE3D1E9
:105AB0004460BDE8F0814261B5E74261D9E700BFCB
:105AC00001617047416170474FF00F0C01F0FC031A
:105AD00003F1804303F5803301F003019A688900E4
:105AE0000CFA01FC22EA0C029A609A688840104382
:105AF00098607047034A536823F44043034353605C
:105B0000704700BF001002401E4A10B4536803F0F3
:105B10000C03082B21D01C4A13460260194A1B4C67
:105B20005168C1F30311615CCB4043605168C1F31C
:105B30000221615C23FA01F181605168C1F3C22145
:105B4000645C1349E340C360526810BCC2F3813205
:105B50008A5CB3FBF2F30361704753685168C3F387
:105B60008343C90303F1020307D55268920304D4A7
:105B7000054A02FB03F30360D0E7064A02FB03F386
:105B80000360CBE70010024000127A008000002082
:105B90007C00002000093D00044A936911B11843BC
:105BA0009061704723EA0000906170470010024046
:105BB000044AD36911B11843D061704723EA000049
:105BC000D061704700100240044AD36811B11843F5
:105BD000D060704723EA0000D06070470010024098
:105BE000044A136911B118431061704723EA000099
:105BF000106170470010024030B504460D46238AFC
:105C0000CA889BB223F4405313438A892382A38911
:105C1000898823F4B05323F00C031B041B0C0B43A3
:105C2000298987B00B43698901A80B439BB2A381E3
:105C3000A38A9BB223F440731343A382FFF764FF4C
:105C4000DDE90332184919488C4208BF1346A2897E
:105C500003EB830312F4004F2A6803EB830314BFA2
:105C600052009200B3FBF2F36425A0FB0321490923
:105C700005FB11330A01A18909040AD41B0132333F
:105C8000A0FB0313C3F3431313439BB2238107B059
:105C900030BDDB003233A0FB0313C3F342131343C5
:105CA0009BB2238107B030BD003801401F85EB5106
:105CB000838921B19BB243F400538381704723F45D
:105CC00000531B041B0C8381704700BF012301F0AC
:105CD0001F0CC1F34211012903FA0CF30DD0022964
:105CE0000CBF103014301AB10268134303607047C0
:105CF000026822EA0303036070470C30F3E700BF39
:105D0000C1F30801818070478088C0F308007047A4
:105D1000C94389B2018070470123C1F3421201F0E7
:105D20001F0C012A03FA0CF313D0022A0CBF028ABB
:105D3000828A92B21340028892B243B10123090AC7
:105D400003FA01F10A4214BF1846002070471846B2
:105D50007047828992B21340EDE700BF0123090A20
:105D60008B40DB439BB20380704700BF08B5174BE5
:105D7000984206D0164B98420FD0164B984218D036
:105D800008BD01214FF40070FFF71EFFBDE8084079
:105D900000214FF40070FFF717BF01214FF480601E
:105DA000FFF712FFBDE8084000214FF48060FFF7C5
:105DB0000BBF01214FF40040FFF706FFBDE808408C
:105DC00000214FF40040FFF7FFBE00BF0024014058
:105DD00000280140003C0140436891F804C023F4CE
:105DE000702310B423F480730C6843EA0C2323431C
:105DF000436083680A4A91F805C01A40D1E902431A
:105E00002343134343EA4C0383600A7CC36A013A89
:105E100023F47003D2B243EA025310BCC36270474A
:105E2000FDF7F1FF836819B143F001038360704708
:105E300023F0010383607047836843F008038360A5
:105E4000704700BF8068C0F3C0007047836843F0AC
:105E500004038360704700BF8068C0F38000704710
:105E600083793BB31D4B01681A6810B422EA010222
:105E70001A605A6822EA01025A60027902F18042ED
:105E800002F582321468214311609968026821EAA0
:105E900002019960D96821EA0201D960417910298B
:105EA00013D001F1804303F58233196810BC0A4313
:105EB0001A6070470379016803F1804303F5823368
:105EC0001A6822EA01021A607047996810BC1143EF
:105ED0009960D9680A43DA60704700BF0004014046
:105EE000054B024619685B69184003D0114214BF84
:105EF00001200020704700BF00040140014B5861A1
:105F0000704700BF0004014010B5B0F820E0204CFD
:105F10002EF0010E4FEA0E4E4FEA1E4EA0F820E082
:105F2000B0F818C042EA03122CF0F30C4FEA0C4C04
:105F3000038C4FEA1C4C4CEA020CA0421FFA8CFC6A
:105F40009BB21BD0134A904218D0B0F1804F15D0AD
:105F5000A2F59832904211D002F5806290420DD0A5
:105F600002F58062904209D023F00A0241EA02035E
:105F700043F00103A0F818C0038410BD23F002030E
:105F80000B4343F00103A0F818C0038410BD00BF09
:105F9000002C01400034014040F6FF4C120242EA5E
:105FA0000333028C10B422F010021204120C02848B
:105FB000028B1A4C0CEA020C4CEA030C038CA04234
:105FC0009AB24FEA01131FFA8CFC9BB21CD004F565
:105FD0000064A04218D0B0F1804F15D0A4F59834D9
:105FE000A04211D004F58064A0420DD004F5806475
:105FF000A04209D022F0A0030B4343F01003A0F805
:1060000018C010BC0384704722F02002134343F0F1
:106010001003A0F818C010BC03847047002C014086
:1060200008B57C4B984242D0B0F1804F4BD07A4BB0
:10603000984252D0794B98422FD0794B984256D003
:10604000784B98425DD0784B984264D0774B984219
:1060500000F08380764B984267D0764B984200F0F0
:106060008880754B984200F09080744B984200F005
:106070009880734B984200F09E80724B984200F0DB
:10608000A480714B984200F0AC80704B984258D07D
:106090006F4B984200F0B18008BD01210420FFF74A
:1060A0009FFDBDE8084000210420FFF799BD0121B4
:1060B0004FF40060FFF788FDBDE8084000214FF471
:1060C0000060FFF781BD01210846FFF789FDBDE8AB
:1060D000084000210120FFF783BD01210220FFF7C6
:1060E0007FFDBDE8084000210220FFF779BD0121B6
:1060F0000820FFF775FDBDE8084000210820FFF7E4
:106100006FBD01211020FFF76BFDBDE808400021A5
:106110001020FFF765BD01212020FFF761FDBDE8DC
:10612000084000212020FFF75BBD01214FF4002033
:10613000FFF74AFDBDE8084000214FF40020FFF7BB
:1061400043BD01214FF40030FFF73EFDBDE808409C
:1061500000214FF40030FFF737BD01214FF400500C
:10616000FFF732FDBDE8084000214FF40050FFF773
:106170002BBD01214FF48010FFF726FDBDE808403C
:1061800000214FF48010FFF71FBD01214FF40010D4
:10619000FFF71AFDBDE8084000214FF40010FFF79B
:1061A00013BD01214020FFF71BFDBDE80840002181
:1061B0004020FFF715BD01218020FFF711FDBDE84C
:1061C000084000218020FFF70BBD01214FF48070B3
:1061D000FFF706FDBDE8084000214FF48070FFF78F
:1061E000FFBC01214FF48030FFF7EEFCBDE8084012
:1061F00000214FF48030FFF7E7BC01214FF48020ED
:10620000FFF7E2FCBDE8084000214FF48020FFF7D3
:10621000DBBC00BF002C014000040040000800402F
:10622000000C004000100040001400400034014009
:10623000004C014000500140005401400018004053
:10624000001C00400020004000400140004401408C
:1062500000480140274A038890429BB212D002F5C1
:10626000006290420ED0B0F1804F0BD0A2F5983270
:10627000904207D002F58062904203D002F580621E
:10628000904203D14A8823F0700313431A4A904284
:1062900017D002F58062904213D0CA8823F440736D
:1062A0009BB21343B1F804C00380124B0A88984292
:1062B000A0F82CC002850CD10B7A038601238382BF
:1062C000704703808B8883850B8803850123838235
:1062D00070470A4B9842EFD003F540639842EBD0E9
:1062E00003F580639842E7D003F580639842E3D0DA
:1062F000ECE700BF002C01400010004000340140DA
:10630000038C30B523F001031B041B0C0384038CA6
:10631000B1F808E0B0F804C04D88028B23F0020306
:106320001B044EEA050E1C4C1B0C22F0730243EAC0
:106330000E031204B1F800E0120CA0421FFA8CFC0C
:106340009BB242EA0E020FD004F50064A0420BD0CB
:1063500004F54064A04207D004F58064A04203D055
:1063600004F58064A04210D14C8923F00803234334
:10637000CD898C892CF4407C2C434CEA040C8C880D
:1063800023F004031FFA8CFC2343C988A0F804C03F
:1063900002838186038430BD002C0140038C30B51C
:1063A00023F010031B041B0C0384038CB1F808E0DA
:1063B000B0F804C04D88028B23F020031B044EEA82
:1063C000050E1B0C22F4E64243EA0E13164CB1F8FC
:1063D00000E01204120C42EA0E22A0421FFA8CFCCA
:1063E0009BB292B20AD004F50064A04206D0C988DC
:1063F000A0F804C002830187038430BD4FF6BF7448
:106400004D8923F0800343EA05131C40CD898B8915
:106410002CF4406C2B434CEA830C8B881FFA8CFCC9
:1064200044EA03139BB2E2E7002C0140038C30B531
:1064300023F480731B041B0C0384038CB1F808E065
:10644000B0F804C04D88828B23F400731B044EEA1D
:10645000050E194C1B0C22F0730243EA0E231204A2
:10646000B1F800E0120CA0421FFA8CFC9BB242EA89
:106470000E020AD004F50064A04206D0C988A0F834
:1064800004C082838187038430BD4FF6FF344D8979
:1064900023F4006343EA05231C40CD898B892CF447
:1064A000405C2B434CEA031C8B881FFA8CFC44EAAB
:1064B00003239BB2E2E700BF002C0140038C30B500
:1064C00023F480531B041B0C0384038CB1F808E0F5
:1064D000B0F804C04D88828B23F400531B044EEAAD
:1064E000050E1B0C22F4E64243EA0E33104CB1F8C1
:1064F00000E01204120C42EA0E22A0421FFA8CFCA9
:106500009BB292B20BD004F50064A04207D0C988B8
:10651000A0F804C08283A0F84010038430BD8C89A9
:106520002CF4804C4CEA841C1FFA8CFCEFE700BF73
:10653000002C01400B8870B50D460446002B4FD04F
:10654000042B00F0A280082B48885AD02B89898818
:106550001B0343EA012140F6FF43228C544E22F4F0
:1065600080521204120C2284A28BB44203EA02036A
:10657000228C43EA01034FEA00319BB292B289B206
:1065800019D006F50066B44215D0B4F1804F12D090
:10659000A6F59836B4420ED006F58066B4420AD00D
:1065A00006F58066B44206D047F6FF510A40024322
:1065B00042F4805204E022F40052114341F480522C
:1065C000A3832284A28BE98822F440621204120C75
:1065D000A283A38B9BB243EA01239BB2A38370BD2A
:1065E0000B898A884988FFF78FFC038BEA8823F0A0
:1065F0000C031B041B0C0383038B9BB21343038309
:1066000070BD228C8B8822F480721204120C0989CE
:106610002284A28B264E92B222F0F3021343228CE4
:1066200043EA0113B4424FEA00219BB292B289B20D
:1066300018D006F50066B44214D0B4F1804F11D0E2
:10664000A6F59836B4420DD006F58066B44209D05E
:1066500006F58066B44205D022F42062024342F47B
:10666000807204E022F40072114341F48072A3832B
:106670002284A38BEA8823F00C031B041B0CA38346
:10668000A38B9BB21343A38370BD0B898A8849886F
:10669000FFF782FC028BE98822F440621204120C9C
:1066A0000283038B9BB243EA01239BB2038370BD39
:1066B000002C014000234FF6FF7203808280C380CC
:1066C00043800372704700BF0023038043808380B0
:1066D000C380038143818381C381704700230122EA
:1066E000038043808280C38003817047038821B187
:1066F0009BB243F001030380704723F001031B04A6
:106700001B0C0380704700BF83899BB212B11943F1
:106710008181704723EA01018181704710B5B0F88B
:1067200008E0B0F818C02EF0070E4FEA0E4E4FEA00
:106730001E4E4EEA0104B0F820E02CF4407C2CF010
:10674000030C2EF022014FEA0C4C090442EA03121A
:106750004FEA1C4C090C4CF4807C11434CF0010CAA
:1067600089B20481A0F818C0018410BD038821B14A
:106770009BB243F080030380704723F080031B0427
:106780001B0C0380704700BF038B23F008031B041E
:106790001B0C0B4303837047038B23F400631B0420
:1067A0001B0C43EA01239BB203837047838B23F0C6
:1067B00008031B041B0C0B4383837047838B23F458
:1067C00000631B041B0C43EA01239BB283837047C5
:1067D00081847047C94389B201827047038A8289E4
:1067E00011EA030092B203D00A4214BF0120002034
:1067F000704700BFC94389B20182704708B50D4B8D
:10680000012198420AD04FF48000FFF7E9F9BDE872
:10681000084000214FF48000FFF7E2B94FF4001068
:10682000FFF7DEF9BDE8084000214FF40010FFF744
:10683000D7B900BF0054004070B504460D4686B07D
:1068400001A8A688FFF760F90398304A26F03F06B2
:10685000A2FB00323604360C46EA9246A680218816
:106860002B682B4E21F001010904090CB342218051
:106870004FEA924123D85B00B0FBF3F30A469BB288
:10688000042B38BF042301322284A3832288A988E1
:1068900092B242F00102228023886A8923F4816344
:1068A00023F00203288911431B04AA891B0C02430D
:1068B0000B439BB292B22380228106B070BD4BF68F
:1068C000FF72EE8896421AD003EB830303EB830337
:1068D000B0FBF3F39BB243F48043C3F30B020AB95A
:1068E00043F001034FF4967000FB01F1094A43F4B1
:1068F0000043A2FB0121890901312184C5E703EB93
:106900004303B0FBF3F39BB2E7E700BF83DE1B4317
:10691000A0860100D34D6210038821B19BB243F0E1
:1069200001030380704723F001031B041B0C038049
:10693000704700BF038821B19BB243F4807303808A
:10694000704723F480731B041B0C0380704700BF47
:10695000038821B19BB243F400730380704723F492
:1069600000731B041B0C0380704700BF038821B118
:106970009BB243F480630380704723F480631B045D
:106980001B0C0380704700BF01827047008AC0B2B1
:10699000704700BF22B141F0010189B20182704706
:1069A00001F0FE0189B20182704700BF838A008B2B
:1069B0009BB243EA00430B4023F07F43581AB0FADE
:1069C00080F04009704700BF002103E00B4B5B588B
:1069D000435004310A480B4B42189A42F6D30A4AF4
:1069E00002E0002342F8043B084B9A42F9D3FEF739
:1069F00035FFF9F7C1FBFBF7EBFFFEE7C06B0008C3
:106A00000000002090000020900000207015002061
:106A1000FEE70000F8B500BFF8BC08BC9E46704712
:0C6A2000F8B500BFF8BC08BC9E467047EB
:106A2C000400002000000000000000000000000036
:106A3C00000000000000000000000000000000004A
:106A4C00000000000000000000000000000000003A
:106A5C00000000000000000000000000000000002A
:106A6C00000000000000000000000000000000001A
:106A7C00000000000000000000000000000000000A
:106A8C00000000004F4B00004B4F00005B25755D74
:106A9C0020416E206572726F72206F636375727223
:106AAC006564207768696C652072756E6E696E67B7
:106ABC002073656C6674657374202872633D25645D
:106ACC002900000020202D20416363656C20583A7A
:106ADC002025730020202D20416363656C20593ADA
:106AEC002025730020202D20416363656C205A3AC9
:106AFC002025730020202D204779726F20583A20D2
:106B0C002573000020202D204779726F20593A20E0
:106B1C002573000020202D204779726F205A3A20CF
:106B2C00257300005B25755D204779726F207365B6
:106B3C006C662D746573742061726520696E636F69
:106B4C006D706C6574652E0071020000E20400002B
:106B5C00C40900008813000010270000204E00001C
:106B6C00409C0000803801000071020000E204002B
:106B7C00232D302B20000000686C4C0065666745A7
:106B8C0046470000303132333435363738394142DC
:106B9C00434445460000000030313233343536373B
:0C6BAC0038396162636465660000000017
:046BB8005901000877
:046BBC00310100089B
:106BC0000400002000000000706A0008506A0008FD
:106BD000306A000800000000000000000000000013
:106BE00000000000000000000000000000000000A5
:106BF0000000000000000000000000000000000095
:106C00000000000000000000000000000000000084
:106C10000000000000000000000000000000000074
:106C200000000000010000000000803F6F12033BE5
:106C3000CDCC4C3F000000000000803F020406085D
:106C40000000000001020304010203040607080912
:04000005080069C9BD
:00000001FF
